:100000004BC0000042C2000040C200003EC20000DF
:100010003CC200000C949E4938C2000036C2000069
:1000200034C2000032C200000C9494490C948A49F6
:100030002CC200002AC2000028C2000026C2000014
:1000400024C2000022C2000020C200001EC2000024
:100050001CC200000C944A4A18C2000016C20000DC
:1000600014C2000012C2000010C200000EC2000044
:100070000CC200000AC2000008C2000006C2000054
:1000800004C2000002C2000000C20000FEC1000065
:10009000FCC10000FAC1000011241FBECFEFD0E266
:1000A000DEBFCDBF0E9400F0D7C10000076342361B
:1000B000B79BD8A71A39685618AEBAAB558C1D3CF9
:1000C000B7CC5763BD6DEDFD753EF6177231BF00BD
:1000D0000000803F05A84CCDB2D44EB93836A902F5
:1000E0000C50B9918688083CA6AAAA2ABE00000036
:1000F000803F08000000BE922449123EABAAAA2A03
:10010000BECDCCCC4C3E00000080BEABAAAAAA3E1D
:1001100000000000BF000000803F00000000000859
:100120004178D3BB4387D1133D190E3CC3BD4282F6
:10013000AD2B3E68EC8276BED98FE1A93E4C80EFB4
:10014000FFBE01C4FF7F3F0000000000FF004C8A9B
:1001500097509545406BA6D8E4B2282EAE90BF26A6
:10016000B14EE86FD0FBE0709A51862C379845323B
:10017000539D06840D971A8CE61E2E0DB41D401655
:100180009AC591F9F786A142660620AFAE19EE270F
:10019000C2BB0EBAB90AAA95CA45040444C1796A19
:1001A00091EE7D3E2E4C960BA96E5A6A9FF56D0519
:1001B000BB8F808DB4F54FC14AE99E674536394FF4
:1001C00075ADF44CB227A939D78036F7C49C7E6A46
:1001D000605F677992B4DD0E4786CD1A6DC6258AB9
:1001E000F464D953D154DB67F78B22BD5CFEA44D78
:1001F000F9A7590EC57E3BF9BA7D430AD39F6C3BE4
:100200000BDEB2875E3710ECC8A6856546290CF177
:10021000D6BCA38C755E4934200DFAE9D7C7B6A7C2
:10022000988A7C6E6155493D32271D1209FFF6EE12
:10023000E5DDD5CEC6BFB9B2ACA6A09A958F8A85AA
:10024000817C78736F6B6864605D5A56FF59E97DF5
:1002500015B150F39942EE9D4F04BC7632F1B2765F
:100260003B03CC98653405D8AC8259320CE7C4A264
:100270008161432509EDD3B9A089725C46321E0B1A
:10028000F8E6D5C4B4A596887A6D6053473C30260D
:100290001B1108FEF5EDE4DCD4CDC6BFB8B1ABA5AB
:1002A0009F99948F8A85807C77736F6B6763605D9D
:1002B000595653504D4A484543403E3C3A383634EF
:1002C00032302E2D2B2A282725242321201F1E1DC6
:1002D0001C1B1A19181716161514131312111110C6
:1002E0000F0F0E0E0D0D0C0C0B0B0B0A0A09090952
:1002F0000808080807070706060606060505050597
:1003000005040404040404030303030303030302B6
:1003100002020202020202020202010101010101C3
:1003200001010101010101010101010101000000C0
:1003300000000000000000000000000000000000BD
:10034000000000000000000000000000FF0C0B0B8C
:100350000B0A0A090909080808080707070606061C
:100360000606050505050504040404040403030347
:100370000303030303020202020202020202020258
:10038000010101010101010101010101010101015D
:10039000010101000000000000000000000000005A
:1003A000000000000000000000000000000000004D
:1003B000000000000000000000000000000000003D
:1003C000000000000000000000000000000000002D
:1003D000000000000000000000000000000000001D
:1003E000000000000000000000000000000000000D
:1003F00000000000000000000000000000000000FD
:1004000000000000000000000000000000000000EC
:1004100000000000000000000000000000000000DC
:1004200000000000000000000000000000000000CC
:1004300000000000000000000000000000000000BC
:1004400000000000000000000000000011241FBE9A
:10045000CFEFD0E2DEBFCDBF1AE1A2ECB9E001C020
:100460001D92A836B107E1F719E0A0E0B1E0E4EE93
:10047000FDEA00E00BBF02C007900D92A23CB1075D
:10048000D9F70E94834A0C94F056BACD2F923F922E
:100490004F925F926F927F928F929F92AF92BF9294
:1004A000CF92DF92EF92FF920F931F93CF93DF9340
:1004B000CDB7DEB727970FB6F894DEBF0FBECDBF1E
:1004C00086E392E10E94BB1440906712509068123C
:1004D0002091001320FF19C025FD02C00C94070DC8
:1004E000420124FD13C080914C1290914D129595BC
:1004F0008795480E591E21FD0BC0C12CD12C7601C9
:1005000022FD10C00FEF1FEF1BC0420121FFF5CFEE
:10051000C0904C12D0904D12EE24D7FCE094FE2CEB
:1005200022FFF0CF009146121091471216950795C1
:100530000095109580914C1290914D12080F191F43
:100540008091211390912213A0E0B0E09058A1096E
:10055000B1091C018091FC12882311F40C94030D45
:100560008091331390913413A0E0B0E09058A1092A
:10057000B109B7FF02C00C94BE0DB595A79597952C
:1005800087959C838B832FB72D83F8948EE390E11E
:100590000E94A23340916210509163105A834983A4
:1005A000AA2497FCA094BA2C662457FC6094762C5D
:1005B0008091781290917912A3019201280F391F2E
:1005C000411D511DDA01C901009731E0A307B105B2
:1005D00024F08FEF9FEFA0E0B0E0B7FF02C00C94D3
:1005E000110D0E94940E46EC41BB469A31E035B99C
:1005F00025E428B950EF5BB992EA9EB987E881BB40
:1006000000C000C041BB469A35B928B960ED6BB94E
:100610009EB981BB00C000C041BB469A35B928B91C
:100620005BB99EB981BB4B815C8169817A81AA27C4
:10063000469FB12D5703C001749FB00D811D9A1FB5
:1006400056039A0BB00D811D9A1F1124AA2797FDFE
:10065000A095BA2F880D991DAA1DBB1D20916C1263
:1006600030916D12820F931FA11DB11D009771E093
:10067000A707B10524F08FEF9FEFA0E0B0E0B7FF30
:1006800002C00C94160D0E94940E46EC41BB469A93
:1006900031E035B921E428B950EF5BB990EA9EB951
:1006A00087E881BB00C000C041BB469A35B928B974
:1006B00060ED6BB99EB981BB00C000C041BB469ADA
:1006C00035B928B95BB99EB981BB910149815A817D
:1006D000AA27249FB12D3503C001529FB00D811D63
:1006E0009A1F34039A0BB00D811D9A1F1124AA275B
:1006F00097FDA095BA2F8C0D9D1DAE1DBF1D20919D
:10070000841230918512820F931FA11DB11D40915B
:10071000B4125091B51260E070E0481759076A07AB
:100720007B0714F00C94BF0BDB01CA010E94940EEE
:1007300046EC41BB469A31E035B921E428B950EF87
:100740005BB992EA9EB987E881BB00C000C041BB9B
:10075000469A35B928B960EE6BB99EB981BB00C025
:1007600000C041BB469A35B928B95BB99EB981BB77
:100770008AE391E10E94A23320915E1130915F11D2
:10078000AA27209FB12D319FC001129FB00D811D5E
:100790009A1F309FB00D811D9A1F1124A0E0B0E078
:1007A0000097A105B10509F4E7C79D5FAF4FBF4FA3
:1007B000009751E0A507B10524F08FEF9FEFA0E06F
:1007C000B0E00E94940E46EC41BB469A31E035B948
:1007D00025E428B950EF5BB990EA9EB987E881BB60
:1007E00000C000C041BB469A35B928B960EB6BB96F
:1007F0009EB981BB00C000C041BB469A35B928B93B
:100800005BB99EB981BB6D816FBF7FB77983F89467
:1008100088E690E10E94A23320918C1030918D10D7
:100820003F832E8380917A1290917B12B301A201B3
:10083000480F591F611D711D4115510531E06307B6
:10084000710524F04FEF5FEF60E070E0DB01CA015B
:1008500077FF02C00C94BD0C0E94940E46EC41BB85
:10086000469A31E035B927E428B950EF5BB992EAEE
:100870009EB987E881BB00C000C041BB469A35B92C
:1008800028B960ED6BB99EB981BB00C000C041BB07
:10089000469A35B928B95BB99EB981BB6B817C8119
:1008A0002E813F81AA27629FB12D7303A001369F3D
:1008B000B00D411D5A1F72035A0BB00D411D5A1F36
:1008C0001124662757FD6095762F480D591D6A1D26
:1008D0007B1D80916E1290916F12480F591F611D00
:1008E000711D4115510531E06307710524F04FEF8B
:1008F0005FEF60E070E0DB01CA0177FF02C00C949B
:10090000DE0C0E94940E46EC41BB469A31E035B9AC
:1009100023E428B950EF5BB990EA9EB987E881BB20
:1009200000C000C041BB469A35B928B960ED6BB92B
:100930009EB981BB00C000C041BB469A35B928B9F9
:100940005BB99EB981BBB1012E813F81AA27629F0D
:10095000B12D7303A001369FB00D411D5A1F7203C4
:100960005A0BB00D411D5A1F1124662757FD609583
:10097000762F4C0D5D1D6E1D7F1D8091861290910E
:100980008712480F591F611D711D8091B6129091F9
:10099000B712A0E0B0E084179507A607B70734F0B8
:1009A00077FF02C00C94ED0CDB01CA010E94940E8B
:1009B00046EC41BB469A31E035B923E428B950EF03
:1009C0005BB992EA9EB987E881BB00C000C041BB19
:1009D000469A35B928B960EE6BB99EB981BB00C0A3
:1009E00000C041BB469A35B928B95BB99EB981BBF5
:1009F00084E691E10E94A2332091881130918911FF
:100A0000AA27209FB12D319FC001129FB00D811DDB
:100A10009A1F309FB00D811D9A1F1124A0E0B0E0F5
:100A20000097A105B10509F4A4C69D5FAF4FBF4F64
:100A3000009731E0A307B10524F08FEF9FEFA0E00E
:100A4000B0E00E94940E46EC41BB469A31E035B9C5
:100A500027E428B950EF5BB990EA9EB987E881BBDB
:100A600000C000C041BB469A35B928B960EB6BB9EC
:100A70009EB981BB00C000C041BB469A35B928B9B8
:100A80005BB99EB981BB49814FBF3FB73983F894A9
:100A900082E990E10E94A2334091B6105091B710C4
:100AA0005F834E8380917C1290917D12B301A201ED
:100AB000480F591F611D711D4115510581E06807DF
:100AC000710524F04FEF5FEF60E070E0DB01CA01D9
:100AD00077FF01C057C70E94940E46EC41BB469A6F
:100AE00031E035B921E428B950EF5BB990EA9EB9FD
:100AF00087E881BB00C000C041BB469A35B928B920
:100B000060EE6BB99EB981BB00C000C041BB469A84
:100B100035B928B95BB99EB981BB2B813C816E8107
:100B20007F81AA27269FB12D3703A001729FB00DA8
:100B3000411D5A1F36035A0BB00D411D5A1F112477
:100B4000662757FD6095762F480D591D6A1D7B1D40
:100B50008091701290917112480F591F611D711D83
:100B60004115510581E06807710524F04FEF5FEFF3
:100B700060E070E0DB01CA0177FD25C70E94940E9A
:100B800046EC41BB469A31E035B925E428B950EF2F
:100B90005BB990EA9EB987E881BB00C000C041BB49
:100BA000469A35B928B960ED6BB99EB981BB00C0D2
:100BB00000C041BB469A35B928B95BB99EB981BB23
:100BC00091016E817F81AA27269FB12D3703A00155
:100BD000729FB00D411D5A1F36035A0BB00D411DB7
:100BE0005A1F1124662757FD6095762F4C0D5D1D09
:100BF0006E1D7F1D8091881290918912480F591F98
:100C0000611D711D8091B8129091B912A0E0B0E001
:100C100084179507A607B70724F077FDD8C6DB0130
:100C2000CA010E94940E46EC41BB469A31E035B9A8
:100C300025E428B950EF5BB992EA9EB987E881BBF9
:100C400000C000C041BB469A35B928B960EE6BB907
:100C50009EB981BB00C000C041BB469A35B928B9D6
:100C60005BB99EB981BB8091921190919311A09133
:100C70009411B09195118B2F9927AA27BB27892B07
:100C80008A2B8B2B09F0F8C58091B711823009F4BB
:100C90009BC508F093C5813009F460C680E090E000
:100CA0006091B0117091B1110E9485142091AE1124
:100CB0003091AF11280F391F3093B3112093B21127
:100CC00080918E1190918F11A0919011B0919111FE
:100CD00040919211509193116091941170919511DE
:100CE000840F951FA61FB71F8093921190939311A5
:100CF000A0939411B0939511AA27209FB12D319FF5
:100D0000C001129FB00D811D9A1F309FB00D811D33
:100D10009A1F1124A0E0B0E00097A105B10509F4E5
:100D200025C59D5FAF4FBF4F009771E0A707B10585
:100D300024F08FEF9FEFA0E0B0E0F6D746EC41BB88
:100D4000469A31E035B921E428B950EF5BB992EA0F
:100D50009EB987E881BB00C000C041BB469A35B947
:100D600028B960EB6BB99EB981BB00C000C041BB24
:100D7000469A35B928B95BB99EB981BB39813FBF65
:100D80003FB73983F8948091C0109091C110A09121
:100D9000C210B091C3108B2F9927AA27BB27892B8C
:100DA0008A2B8B2B09F07CC58091E510823009F4E9
:100DB00022C508F01AC5813009F4C1C580E090E071
:100DC0006091DE107091DF100E9485144091DC105C
:100DD0005091DD10480F591F5F834E835093E110EF
:100DE0004093E0108091BC109091BD10A091BE1076
:100DF000B091BF104091C0105091C1106091C210CD
:100E00007091C310840F951FA61FB71F8093C01049
:100E10009093C110A093C210B093C31080917E1222
:100E200090917F12B301A201480F591F611D711DDE
:100E30004115510581E06807710524F04FEF5FEF20
:100E400060E070E0DB01CA0177FDACC56DD766ECF0
:100E500061BB469A51E055B943E448B970EF7BB99C
:100E600090EA9EB987E881BB00C000C061BB469A8A
:100E700055B948B9E0EEEBB99EB981BB00C000C0DE
:100E800061BB469A55B948B97BB99EB981BB2B81E4
:100E90003C816E817F81AA27269FB12D3703A00157
:100EA000729FB00D411D5A1F36035A0BB00D411DE4
:100EB0005A1F1124662757FD6095762F480D591D3E
:100EC0006A1D7B1D8091721290917312480F591FF9
:100ED000611D711D4115510581E06807710524F000
:100EE0004FEF5FEF60E070E0DB01CA0177FD56C5B0
:100EF0001BD766EC61BB469A51E055B947E448B947
:100F000070EF7BB990EA9EB987E881BB00C000C052
:100F100061BB469A55B948B9E0EDEBB99EB981BBC2
:100F200000C000C061BB469A55B948B97BB99EB9AB
:100F300081BB91016E817F81AA27269FB12D370346
:100F4000A001729FB00D411D5A1F36035A0BB00D00
:100F5000411D5A1F1124662757FD6095762F4C0DB1
:100F60005D1D6E1D7F1D80918A1290918B12480F1E
:100F7000591F611D711D8091BA129091BB12A0E0A2
:100F8000B0E084179507A607B70724F077FD2CC5B6
:100F9000DB01CA01C9D646EC41BB469A31E035B9FE
:100FA00027E428B950EF5BB992EA9EB987E881BB84
:100FB00000C000C041BB469A35B928B960EE6BB994
:100FC0009EB981BB00C000C041BB469A35B928B963
:100FD0005BB99EB981BB8091BC119091BD11A0916C
:100FE000BE11B091BF118B2F9927AA27BB27892B40
:100FF0008A2B8B2B09F04AC48091E111823009F4CD
:101000002AC408F022C4813009F454C480E090E07E
:101010006091DA117091DB110E9485142091D81132
:101020003091D911280F391F3093DD112093DC1135
:101030008091B8119091B911A091BA11B091BB11E2
:101040004091BC115091BD116091BE117091BF11C2
:10105000840F951FA61FB71F8093BC119093BD11DD
:10106000A093BE11B093BF11AA27209FB12D319F2D
:10107000C001129FB00D811D9A1F309FB00D811DC0
:101080009A1F1124A0E0B0E00097A105B10509F472
:101090006AC39D5FAF4FBF4F009771E0A707B105CF
:1010A00024F08FEF9FEFA0E0B0E03ED646EC41BBCE
:1010B000469A31E035B923E428B950EF5BB992EA9A
:1010C0009EB987E881BB00C000C041BB469A35B9D4
:1010D00028B960EB6BB99EB981BB00C000C041BBB1
:1010E000469A35B928B95BB99EB981BB39813FBFF2
:1010F0002FB72983F8948091EA109091EB10A0917A
:10110000EC10B091ED108B2F9927AA27BB27892BC4
:101110008A2B8B2B09F0B5C380910F11823009F413
:1011200081C308F079C3813009F4D3C380E090E033
:1011300060910811709109110E9485144091061167
:1011400050910711480F591F5F834E8350930B1125
:1011500040930A118091E6109091E710A091E81059
:10116000B091E9104091EA105091EB106091EC10B1
:101170007091ED10840F951FA61FB71F8093EA1082
:101180009093EB10A093EC10B093ED10809180122F
:1011900090918112B301A201480F591F611D711D69
:1011A0004115510581E06807710524F04FEF5FEFAD
:1011B00060E070E0DB01CA0177FDF8C3B5D566ECED
:1011C00061BB469A51E055B945E448B970EF7BB927
:1011D00090EA9EB987E881BB00C000C061BB469A17
:1011E00055B948B9E0EEEBB99EB981BB00C000C06B
:1011F00061BB469A55B948B97BB99EB981BB2B8171
:101200003C816E817F81AA27269FB12D3703A001E3
:10121000729FB00D411D5A1F36035A0BB00D411D70
:101220005A1F1124662757FD6095762F480D591DCA
:101230006A1D7B1D8091741290917512480F591F81
:10124000611D711D4115510581E06807710524F08C
:101250004FEF5FEF60E070E0DB01CA0177FDAAC3EA
:1012600063D566EC61BB469A51E055B941E448B993
:1012700070EF7BB992EA9EB987E881BB00C000C0DD
:1012800061BB469A55B948B9E0EDEBB99EB981BB4F
:1012900000C000C061BB469A55B948B97BB99EB938
:1012A00081BB91016E817F81AA27269FB12D3703D3
:1012B000A001729FB00D411D5A1F36035A0BB00D8D
:1012C000411D5A1F1124662757FD6095762F4C0D3E
:1012D0005D1D6E1D7F1D80918C1290918D12480FA7
:1012E000591F611D711D8091BC129091BD12A0E02B
:1012F000B0E084179507A607B70724F077FD6AC307
:10130000DB01CA0111D546EC41BB469A31E035B943
:1013100021E428B950EF5BB990EA9EB987E881BB18
:1013200000C000C041BB469A35B928B960EB6BB923
:101330009EB981BB00C000C041BB469A35B928B9EF
:101340005BB99EB981BB82EE91E10E94A2332091EC
:10135000061230910712AA27209FB12D319FC0019C
:10136000129FB00D811D9A1F309FB00D811D9A1FD5
:101370001124A0E0B0E00097A105B10509F4F0C187
:101380009D5FAF4FBF4F009771E0A707B10524F0F5
:101390008FEF9FEFA0E0B0E0C7D446EC41BB469A88
:1013A00031E035B925E428B950EF5BB992EA9EB92E
:1013B00087E881BB00C000C041BB469A35B928B957
:1013C00060EB6BB99EB981BB00C000C041BB469ABF
:1013D00035B928B95BB99EB981BB29812FBF3FB709
:1013E0003D83F89480E191E10E94A2334091341151
:1013F000509135115A8349838091821290918312C2
:10140000480E591E611C711C4114510451E06506BF
:1014100071042CF044244A94542C612C712CD30177
:10142000C20177FCB3C280D446EC41BB469A31E09E
:1014300035B927E428B950EF5BB990EA9EB987E83F
:1014400081BB00C000C041BB469A35B928B960EEE7
:101450006BB99EB981BB00C000C041BB469A35B98B
:1014600028B95BB99EB981BB6B817C8129813A81A6
:10147000AA27629FB12D7303A001369FB00D411DB5
:101480005A1F72035A0BB00D411D5A1F11246627B3
:1014900057FD6095762F480D591D6A1D7B1D809163
:1014A000761290917712480F591F611D711D4115D9
:1014B000510531E06307710524F04FEF5FEF60E005
:1014C00070E0DB01CA0177FD65C22ED446EC41BB5A
:1014D000469A31E035B923E428B950EF5BB992EA76
:1014E0009EB987E881BB00C000C041BB469A35B9B0
:1014F00028B960ED6BB99EB981BB00C000C041BB8B
:10150000469A35B928B95BB99EB981BBB101298129
:101510003A81AA27629FB12D7303A001369FB00DB7
:10152000411D5A1F72035A0BB00D411D5A1F112441
:10153000662757FD6095762F4C0D5D1D6E1D7F1D36
:1015400080918E1290918F12480F591F611D711D4D
:101550008091BE129091BF12A0E0B0E08417950771
:10156000A607B70724F077FD3CC2DB01CA01DCD334
:1015700046EC41BB469A31E035B923E428B950EF37
:101580005BB990EA9EB987E881BB00C000C041BB4F
:10159000469A35B928B960EB6BB99EB981BB00C0DA
:1015A00000C041BB469A35B928B95BB99EB981BB29
:1015B0008091101290911112A0911212B0911312F9
:1015C0008B2F9927AA27BB27892B8A2B8B2B09F0D6
:1015D00062C180913512823009F4DFC008F0D7C0B3
:1015E000813009F49BC180E090E060912E127091EF
:1015F0002F120E94851420912C1230912D12280F49
:10160000391F309331122093301240910C125091B7
:101610000D1260910E1270910F12C0901012D090A6
:101620001112E0901212F09013124C0D5D1D6E1D00
:101630007F1D4093101250931112609312127093F9
:101640001312AA27209FB12D319FC001129FB00D08
:10165000811D9A1F309FB00D811D9A1F1124A0E09B
:10166000B0E00097A105B10509F477C09D5FAF4FC9
:10167000BF4F009731E0A307B10524F08FEF9FEF34
:10168000A0E0B0E051D346EC41BB469A31E035B919
:1016900027E428B950EF5BB992EA9EB987E881BB8D
:1016A00000C000C041BB469A35B928B960EB6BB9A0
:1016B0009EB981BB00C000C041BB469A35B928B96C
:1016C0005BB99EB981BB3D813FBF2091C209922F7A
:1016D0009C7111E009F010E0922F9370923009F4A0
:1016E000AAC1933009F43EC2913009F4AFC111117F
:1016F00050C280E00E94F9418091870D9091880D41
:10170000A091890DB0918A0D0196A11DB11D809304
:10171000870D9093880DA093890DB0938A0D209129
:10172000C2092F5F2093C20927960FB6F894DEBF37
:101730000FBECDBFDF91CF911F910F91FF90EF9022
:10174000DF90CF90BF90AF909F908F907F906F90E1
:101750005F904F903F902F90089580E090E092CF5F
:1017600080E090E019CE80E090E09FCC80E090E0B7
:10177000E4CA80E090E065C980E090E022C8B7FD4F
:1017800002C00C94960380E090E00C9496038330A2
:1017900009F4BFC0843009F026CF60911012709117
:1017A000111280911212909113122091321240E284
:1017B00051E00E94D6258095909517CF833009F48B
:1017C00099C0843009F06ACA6091921170919311A6
:1017D00080919411909195112091B41140E251E0C3
:1017E0000E94D625809590955BCA833009F45DC030
:1017F000843009F0E3CA6091C0107091C1108091EB
:10180000C2109091C3102091E21040E251E00E947A
:10181000D62580959095D4CA833009F475C084305C
:1018200009F084CC6091EA107091EB108091EC107B
:101830009091ED1020910C112111DDC0BB27A92F33
:10184000982F872F8095909573CC833009F457C0DB
:10185000843009F0DBCB6091BC117091BD11809197
:10186000BE119091BF112091DE1140E251E00E9423
:10187000D62580959095CCCB8EE891E10E945D3382
:1018800003CA86EE90E10E945D3346CC88EB91E17D
:101890000E945D33B1CB8CE092E10E945D3399CE22
:1018A0008CEB90E10E945D337FCA8091D0109091C3
:1018B000D11086CA6091BC117091BD118091BE118A
:1018C0009091BF112091DE1140E253E00E94D62595
:1018D0009FCB6091EA107091EB108091EC10909189
:1018E000ED1020910C1121118AC0BB27A92F982F30
:1018F000872F1ECC8091A2119091A311D1C9809104
:10190000CC119091CD1184CB8091FA109091FB1065
:101910000FCC809120129091211267CE609110120D
:101920007091111280911212909113122091321223
:1019300021115DC0BB27A92F982F872F56CE60910C
:10194000C0107091C1108091C2109091C31020916D
:10195000E21040E253E00E94D62532CA6091921113
:101960007091931180919411909195112091B411DF
:1019700040E253E00E94D62593C980E090E0DC016C
:101980000C942C0480E090E0DC01A5C880E090E09D
:10199000DC0149CD80E090E0DC0197CD80E090E073
:1019A000DC01A6CA80E090E0DC0150CA80E090E053
:1019B000DC0104CC80E090E0DC0152CC80E090E0DF
:1019C000DC010C94810480E090E0DC01D7C880E069
:1019D00090E027C980E090E095CC80E090E00C9406
:1019E000D60480E090E0C3CD80E090E0D3CA40E22E
:1019F00053E09CD7FACD40E251E098D723CF40E2A4
:101A000053E094D795CB1C821B820C94C302809028
:101A10004C1290904D1295948794840C951C0C94C4
:101A2000710280E090E0DC010C94F10280E090E033
:101A3000DC010C94430381E592E19DD78091001372
:101A400088700E94E4282091C2096BCE0E94E4397C
:101A50008091A614882309F496C08091F3128823FC
:101A600039F081508093F3120E946C198111BAC031
:101A70008091EC12882309F47EC02091EA12309103
:101A8000EB1200E912E18CE6882E82E1982EA4E8A0
:101A9000B2E168EA72E198E7A92E92E1B92E4CE929
:101AA00052E1D12C42C0E81AF90A2E153F0508F47C
:101AB0007901E80EF91EF401F182E082FA01E19069
:101AC000F190AF01F501808191818E159F0508F09D
:101AD00063C0E81AF90A2E153F0508F47901E80EEB
:101AE000F91EF501F182E082FB01E190F190BF0166
:101AF0008D919C9111978E159F0508F05FC0E81A93
:101B0000F90A2E153F0508F47901E80EF91E119621
:101B1000FC92EE92D394F2E08F0E911C129682E02A
:101B2000A80EB11C96E0D91631F1F801E190F190C0
:101B30008F01F401808191818E159F0508F4B3CF48
:101B4000E816F90608F0BACFFC01EE19FF097F018B
:101B50002E173F0708F479018E199F09F40191832C
:101B60008083ACCF22FDDDCD812F0E943E2A812FC4
:101B700046D2111135C02091C209D3CD0196A11DC5
:101B8000B11D0C94BD028091F312882309F46CCF2F
:101B900068CF0E941934ADCDE816F90608F0A4CF3D
:101BA000FC01EE19FF097F012E173F0708F47901A8
:101BB0008E199F09F5019183808396CFE816F90667
:101BC00008F0A8CFFC01EE19FF097F012E173F078F
:101BD00008F479018E199F0911969C938E939ACFE0
:101BE000AFD5C9CF8091E60B811103C080916E0CF7
:101BF00081110E94473B80917F0D882309F438CFE3
:101C00000E947E3A35CFEAE7F8E180818F5F8083DA
:101C1000089555E05A95F1F7000036EC31BB469A2D
:101C200080EE87B997E09AB98DB915B880E488B984
:101C30001BB880E28EB987E481BB82E08A95F1F718
:101C400000C026B199B18CB131BB479A37EE37B994
:101C500037EF3AB932EE3DB9422F4695437050E81E
:101C6000259F90011124422B292F2071422B292FCF
:101C7000269526952870422B96959076492B90E0D4
:101C8000880F991F84709927842B089536EC20EED5
:101C900097E0A0E8F7E4E7EE77EF62EE5FB7F8943D
:101CA00031BB469A27B99AB92DB915B8A8B99BB9CD
:101CB0001EB8F1BB42E04A95F1F700C046B1B9B198
:101CC000BCB131BB479AE7B97AB96DB95FBF55E08E
:101CD0005A95F1F7000042FFE1CF5FB7F89496EC18
:101CE00091BB469A382F330F982F9695232F267045
:101CF0002068482F441F4427441F242B8071836091
:101D0000432F440F4072842B307C832B927090625F
:101D100015B828B98BB99EB987E881BB85E08A954B
:101D2000F1F700005FBF08959C01232F332726950C
:101D30002695722F66EC61BB469A522F550F452FA0
:101D400046704068207133272260352F330F307280
:101D5000322B507C352B272F26952270206215B808
:101D600048B93BB92EB957E851BB969587959695DA
:101D70008795282F61BB469A482F440F382F3695F8
:101D8000221F2227221F642F6670262B2068807155
:101D900099278260942F990F9072982B407C942BF6
:101DA000327015B828B99BB93EB951BB08952F922E
:101DB0003F924F925F926F927F928F929F92AF92DB
:101DC000BF92CF92DF92EF92FF920F931F93CF9328
:101DD000DF93CDB7DEB728970FB6F894DEBF0FBEFE
:101DE000CDBF8D832FB72E83F894282F2595259569
:101DF0002595259580E290E002C0959587952A95D6
:101E0000E2F79D819F70982B86EC81BB469A492F03
:101E1000440F292F2695392F331F3327331F842F43
:101E20008670382B30649071842F880F8072892BD4
:101E3000407C842B2270206491E095B938B98BB92D
:101E40002EB987E881BB35E03A95F1F700002D8186
:101E5000332727FD30953A832983F901EC5CF94F4C
:101E6000C080D12C80E190E08C199D092FEF3FEFCD
:101E7000082E02C0369527950A94E2F702C0220F79
:101E8000331F8A95E2F73C832B83E12CF12C00E091
:101E900010E82FEF3FEF96ECA92E40EEB42E57E05E
:101EA000252E3324339460E4462E70E2572EE7E467
:101EB0006E2EF7EE7F2EA7EF8A2EB2EE9B2E0AC073
:101EC000200F311F16950795AFEFEA1AFA0ACE14C4
:101ED000DF042CF1C9012F83388726DF82E08A9541
:101EE000F1F700C0A1BA469AB7B82AB8BDB835B85C
:101EF00048B81BB85EB861BA92E09A95F1F700C095
:101F000086B189B19CB1A1BA479A77B88AB89DB811
:101F10002F81388585FDD4CF201B310BD3CF86ECA4
:101F200081BB469A81E085B987E488B980EF8BB997
:101F300082E48EB987E881BBB5E0BA95F1F700007D
:101F4000EB81FC812E233F23E981FA81EE0FFF1FF5
:101F5000ED54F04F31832083232F3327E981FA8119
:101F6000E157F04F848190E0821B930B97FD1DC0D9
:101F7000059704F53E813FBF28960FB6F894DEBF63
:101F80000FBECDBFDF91CF911F910F91FF90EF90CA
:101F9000DF90CF90BF90AF909F908F907F906F9089
:101FA0005F904F903F902F90089591958195910962
:101FB000059704F3248381E090E0A0E0B0E00D8079
:101FC00004C0880F991FAA1FBB1F0A94D2F7409123
:101FD0008F0F5091900F6091910F7091920F842B01
:101FE000952BA62BB72B80938F0F9093900FA093D8
:101FF000910FB093920F2D812093F40FBBCFCF930D
:10200000882339F18091490A8F5F8093490A85318D
:1020100048F081E090914A0A9111CDC080934A0A1C
:102020001092490AC0914D0AC11179C05091470AD6
:102030009091480AE0914E0AE13009F4DEC008F4BC
:10204000AFC0E23009F4C4C020E0F0E0ED5BF54F32
:102050002487AFB7F89456EC51BB469A41E045B996
:1020600080E488B91BB880E28EB937E831BB00C084
:1020700000C080E190E000904E0A02C0880F991FD6
:102080000A94E2F7282F51BB469A782F770F682FD2
:102090006695221F2227221F972F9670292B2064D6
:1020A0008071972F990F9072982B707C972B62708C
:1020B00045B928B99BB96EB931BB00C000C0E091E9
:1020C0004E0AF0E0ED5BF54F848551BB469A582FE0
:1020D000550F982F9695252F26702064682F661F20
:1020E0006627661F262B682F6071852F880F8072E8
:1020F000862B507C852B9270906245B928B98BB99C
:102100009EB931BBAFBF80914E0A90E0019663E06B
:1021100070E00E94E25180934E0ACF910895409161
:102120004B0A4F5F40934B0AE2E5FAE00190002032
:10213000E9F7E355FA4020914C0A332727FD309503
:10214000C90101966E2F772767FD70950E94E251B5
:10215000F901ED5BF54F278530E02038310588F136
:102160005FEFE82FFF27E7FDF095ED5BF54F278543
:1021700030E02038310550F5F901EC5AF94F9081E3
:10218000403108F457CF80934C0A10924B0A8111CA
:1021900051CF1C160CF04ECFC150C0934D0A4ACF00
:1021A0002091430A80914A0A882309F44ECF8091F6
:1021B000450A28274ACF80E080934A0A1092490AAC
:1021C00031CFF901EC5AF94F5081CBCF9FEFD8CFE7
:1021D000292F2F778091430A9091440A90FD20681F
:1021E0008091450A9091460A90FF2FCF80914A0A2C
:1021F000882309F42ACF205828CF252F2F778091C4
:10220000430A9091440A91FD20688091450A90917B
:10221000460A91FF1ACFEACF4FB7F8948091391050
:1022200096EC91BB469A382F330F982F9695232F13
:1022300026702064582F551F5527551F252B582FC2
:102240005071832F880F8072852B307C832B927086
:10225000906631E035B928B98BB99EB987E881BB62
:102260004FBF089596EC91BB469A582F56955695B8
:1022700056958295880F807E462F440F362F3695CF
:10228000242F26702064962F991F9927991F292B98
:102290006071942F990F9072962B407C942B327022
:1022A000832B55B928B99BB98EB987E881BB85E0E6
:1022B0008A95F1F700000895CF93DF93AADCC82F29
:1022C000D0E0A7DC382F20E0C22BD32B60E081E0E8
:1022D000C9DF60E081E0C6DF61E082E0C3DF60E08B
:1022E00082E0C0DFC095D095CE01DF91CF910895F7
:1022F0006095E9E7F8E19081982B6923608386EC8B
:1023000081BB469A362F330F962F9695262F221F84
:102310002227221F832F8670282B20646071832F31
:10232000880F8072862B307C832B9270906C31E00A
:1023300035B928B98BB99EB987E881BB85E08A9504
:10234000F1F70000E8E7F8E180818F5F808308956E
:10235000CF92DF92EF92FF920F931F93CF93DF9371
:1023600090E040E452E46FE070E0F6ECE0EEC7E0AD
:10237000DC2EEE24E394D0E4FD2E00E217E4D7EE49
:10238000C7EFB2EE05C0411551056105710571F148
:10239000F1BB469AE7B9DAB8EDB9E5B8F8B81BB8B9
:1023A0000EB911BB22E02A95F1F700C0A6B1C9B061
:1023B000CCB0F1BB479AD7B9CAB9BDB941505109A0
:1023C00061097109A2FB222720F930E082179307E7
:1023D000D1F6452B462B472B49F0DF91CF911F912A
:1023E0000F91FF90EF90DF90CF900895DF91CF9104
:1023F0001F910F91FF90EF90DF90CF9004CCDF9270
:10240000EF92FF920F931F93CF93DF9390E040E4FE
:1024100052E46FE070E0F6ECE0EE17E0D12EEE242F
:10242000E39400E4F02E00E217E4D7EEC7EFB2EE3B
:1024300005C0411551056105710569F1F1BB469A69
:10244000E7B9DAB8EDB9E5B8F8B81BB80EB911BB01
:1024500022E02A95F1F700C0A6B1A9B1ACB1F1BB59
:10246000479AD7B9CAB9BDB9415051096109710933
:10247000A1FB222720F930E082179307D1F6452BE4
:10248000462B472B41F0DF91CF911F910F91FF9089
:10249000EF90DF900895DF91CF911F910F91FF9002
:1024A000EF90DF90B0CBCF93DF93E0E8FDE0808149
:1024B000C2E8DDE0688190E070E00E94E251A09106
:1024C000830DB091840DA80FB91F2C913FB7F894DC
:1024D000808190E00196688170E00E94E2518083E3
:1024E0003FBF822FDF91CF91D1CB0F931F93072F47
:1024F000069510E00F771127282F2F774091A4140D
:102500004F704069E0917B19F0917C1963E070E0B5
:102510008BE799E109951F910F9108950F93262F4D
:102520004F772F778F708068E0917B19F0917C193D
:10253000042F482F63E070E08BE799E109950F9134
:102540000895EF92FF920F931F93CF93DF93EC01C7
:10255000162FF42EE22E8091A019843071F1C23032
:10256000D10509F453C0C330D10571F1C130D10593
:10257000F9F1C430D105C8F5E0919719F091981997
:10258000309739F00E2D2F2D412FBE018BE799E1A9
:102590000995E0919919F0919A19309739F00E2D1B
:1025A0002F2D412FBE018BE799E10995DF91CF9146
:1025B0001F910F91FF90EF900895E0919519F09180
:1025C00096193097F9F6D8CF862F807F803A09F494
:1025D0008DC008F041C0803809F456C0803961F6DA
:1025E000E0917F19F091801942C0C0E0D0E0C4CFE3
:1025F000683F50F1E0919119F0919219309709F4E8
:10260000BBCF612F8BE799E10995C3CF862F807FE0
:10261000803D09F455C0803F09F440C0803C09F07A
:10262000ABCFE0918919F0918A19309709F4A4CFC2
:10263000133F09F43FC0113FE9F1612F6F704F2D37
:102640008BE799E10995A5CF663F09F095CFE09119
:102650009319F0919419D2CF803ED9F0803FA9F11F
:10266000803B09F089CFE0917D19F0917E19309778
:1026700009F482CF123F99F1612F6F702E2D4F2DEB
:102680008BE799E1099585CFE0918119F091821945
:10269000EECFE0918519F0918619E9CF633F59F1AA
:1026A000613F09F069CFE0918F19F091901930974F
:1026B00009F462CF4F2D612F8BE799E1099569CF1E
:1026C000E0918B19F0918C19B0CF623F09F054CF93
:1026D000E0918719F0918819309709F44DCF2E2D8C
:1026E0004F2D62EF8BE799E1099553CFE091831964
:1026F000F0918419BCCFE0918D19F0918E1930972B
:10270000C9F63ACF21E020934D0A0097A9F0109224
:102710004C0ABC0183E59AE00E94F655E2E5FAE036
:1027200001900020E9F7E355FA40EE5AF54F80E2B8
:1027300090E09183808308958FEF80934C0A0895F1
:1027400080917A13882319F0815080937A13089529
:1027500010928F0F1092900F1092910F1092920F73
:102760008FEF8093F40F80936C138FEF9FEFDC015A
:1027700080936D1390936E13A0936F13B0937013A7
:1027800008958F929F92AF92BF92CF92DF92EF9275
:10279000FF920F931F934A015B0168017901BC010D
:1027A00080E090E00E9426539058A50194010E9479
:1027B00061520E94CE52A70196010E94AA540E9423
:1027C000FA52CB011F910F91FF90EF90DF90CF90C5
:1027D000BF90AF909F908F9008950F931F93E4E860
:1027E000FAE090E02191922B2AE0E439F207D1F748
:1027F00031E0911101C030E0ECE9FBE090E0208194
:10280000922B3C962BE0E43EF207C9F791110BC0E6
:102810004FEF5FEFBA014093ED125093EE126093C9
:10282000EF127093F012332321F09091CE1699237A
:10283000D1F03093CE16882399F080914113909176
:10284000421300E010E42CE135E440E050E86BE393
:1028500076E48095909595DF9093F2128093F11233
:102860001F910F9108954091870D5091880D6091AF
:10287000890D70918A0D4093ED125093EE12609382
:10288000EF127093F012D5CF0F931F93CF93DF9376
:10289000EC018A899B8900E01FEF2FE737E440E0D5
:1028A00050E26BE476E4809590956BDFAC0160E0DC
:1028B00070E0088C04C0440F551F661F771F0A94F0
:1028C000D2F7488759876A877B87DF91CF911F911D
:1028D0000F910895CF93DF93EC017B8B6A8BD4DF4C
:1028E000A98DBB27A1950CF4B095AA0FBB1F11961B
:1028F000288539854A855B850E948D566C877D8742
:102900008E879F87DF91CF910895AC01AA27469FBC
:10291000B12D579F9001749FB00D211D3A1F569FF6
:10292000B00D211D3A1F1124C9010895A72F8F3F13
:10293000F9F0282F2F5F30E0220F331FE82FF0E04F
:10294000EE0FFF1FE40FF51F60817181FA01E20FA6
:10295000F31F80819181861B970B892F9927A89F50
:102960009001A99F300D1124260F371FC90108952A
:102970002EEF31E0E3CF8F929F92AF92BF92CF9232
:10298000DF92EF92FF92CF93DF93EC01CC80DD805A
:10299000EE80FF808F2D9927AA27BB27892B8A2BB2
:1029A0008B2B09F051C08A8D8C849D84AE84BF84AA
:1029B000833009F470C068F5813009F498C08C89BF
:1029C0009D89C80CD91CEA1CFB1CCC82DD82EE82DE
:1029D000FF82BC01705848895989AA27649FB12D8C
:1029E00075039001569FB00D211D3A1F74033A0BD9
:1029F000B00D211D3A1F11242E8B3F8BDF91CF91FB
:102A0000FF90EF90DF90CF90BF90AF909F908F900E
:102A10000895843009F447C0853009F0D0CFB7015C
:102A2000A601E9E07695679557954795EA95D1F720
:102A3000CA015D8B4C8B298D222309F4C2CF80956E
:102A400090959D8B8C8BBDCFE1E0898DE81BE98F44
:102A5000E11155C0C12CD12C7601CC82DD82EE82F1
:102A6000FF82FF27E1950CF4F095DF01AA0FBB1F51
:102A70001196288539854A855B850E948D564B01C4
:102A80005C016C877D878E879F878A8D81113DC011
:102A9000FD8BEC8B94CF4EEC54E1C701B60146DFC1
:102AA0009D8B8C8B8ECF2B8922952F7048815981DD
:102AB0006A817B81972F440F551F661F771F892FCF
:102AC000881F8827881F392F3295369537708327BE
:102AD0008927969589278170482B215058F748837C
:102AE00059836A837B83CA015D8B4C8B6ACF7727BE
:102AF0006F2D5E2D4D2DCA015D8B4C8B62CFCC248A
:102B0000CA94DC2CEC2CF12CA8CF823009F050CFE9
:102B10000E9448567D8B6C8B8A8D8C849D84AE84FC
:102B2000BF84CC80DD80EE80FF8042CFEF92FF92A9
:102B30000F931F93CF93DF93F82EEFB6F89484E7AB
:102B4000E5EFF2E1DF011D928A95E9F780E090E878
:102B5000909314138093131390931A138093191363
:102B60002FEF3FEF30931E1320931D1390932213EA
:102B70008093211330932E1320932D13309312132F
:102B80002093111390933E1380933D1390934A1317
:102B900080934913909344138093431385E080936B
:102BA000081381E080930913809302138093041328
:102BB00080930A1382E080930B1346E050E06FEF9E
:102BC00070E08BE493E10E94E45501E513E1C0E07D
:102BD000D0E0BE01882777FD8095982F0E9428536A
:102BE0002BEA3AEA4AEA55E40E94AA540E94FA52B1
:102BF000F801619371938F012196CC30D10549F78B
:102C0000F11008C0EFBEDF91CF911F910F91FF909F
:102C1000EF90089581E08093F512EFBEDF91CF91A0
:102C20001F910F91FF90EF9008958F929F92AF9216
:102C3000BF92DF92EF92FF920F931F93CF93DF9398
:102C40009C01862E912C8114910409F445C081E0E9
:102C5000881A9108A12CB12CAFEF8A1A9A0AAA0AF5
:102C6000BA0ABA2CA92C982C882480E090E0DC01C8
:102C7000A90160E070E0403E51056105710510F565
:102C80005F5F6F4F7F4F762F652F542F4427FCE8EF
:102C9000EF2EFDE0FF2EE80EF91EC0E0D0E000E0D0
:102CA00010E06BBFFA01D790F701E00FF11FD0825F
:102CB00021968E014F5F5F4F6F4F7F4FC115E1E04F
:102CC000DE0779F72F5F3F4F9F5FAF4FBF4F8815EC
:102CD0009905AA05BB0561F610928E0F80918C0DA7
:102CE00090918D0DA0918E0DB0918F0D20E93DE05A
:102CF00030938D0F20938C0F853A9641A146B105F4
:102D0000B9F42091900D81E99DE090938D0F80930F
:102D10008C0F20938E0F81E0DF91CF911F910F9147
:102D2000FF90EF90DF90BF90AF909F908F900895AD
:102D300080E092E0ECE8FDE0DF019C011D92215073
:102D40003040E1F780E0E8CFEF92FF920F931F93BE
:102D5000CF93DF93E82EEB01FFB6F89461E065DFD7
:102D6000ECE8FEE040E051E004C0A9012115310586
:102D7000F9F09A012150310992919923B1F39A0106
:102D80008A010F5F1F4FE092E116E2EEF6E18CE858
:102D90009DE0A901BC01CF010E94CA551983088397
:102DA000FFBEDF91CF911F910F91FF90EF9008959B
:102DB00001E010E020E030E0E6CF1F93CF93DF93F7
:102DC0001FB7F89461E031DF882309F496C080E0F2
:102DD000ADDE10924B138FEF80934C1380934D1305
:102DE00080934E1380934F138093501330918E0F26
:102DF000332309F47CC0C0918C0FD0918D0F20E05B
:102E000089919991E22FF0E0EE0FFF1FE15FFC4EF8
:102E1000918380832F5F293199F7C0938C0FD093D2
:102E20008D0F80E09991DE01D0938D0FC0938C0FB0
:102E3000E82FF0E0EB50FD4E90838F5F873191F7E4
:102E40008091051380930E13323008F450C08D9199
:102E50009D91E22FF0E0EE0FFF1FE15FFC4E9183AA
:102E600080832F5F2E3199F7B0938D0FA0938C0F35
:102E7000FD018191F0938D0FE0938C0F80930C13E3
:102E800011968C911197ED012296D0938D0FC093DE
:102E90008C0F80930D13EBE4F3E18991D0938D0FA8
:102EA000C0938C0F819383E1E135F807B1F78091EE
:102EB000A9149091AA1490934A1380934913373020
:102EC000B0F0FD013896C1E5D3E1909681919191E2
:102ED00089939993EA17FB07C9F7F0938D0FE09355
:102EE0008C0F1FBF81E0DF91CF911F91089581E08A
:102EF0001FBFDF91CF911F91089580E01FBFF9CFD1
:102F0000ECE8FDE080E092E0DF019C011D922150A1
:102F10003040E1F727E020938E0F85EA96E1A1E6A5
:102F2000B0E080839183A283B383248381E99DE011
:102F300090938D0F80938C0F0895833061F08931C9
:102F400051F08F3141F091E08F3019F0803109F06C
:102F500090E0892F089591E0892F08958F929F9294
:102F6000AF92BF92EF92FF921F93CF93DF93109295
:102F70008B0DC0E0D0E014E26C2F772767FD7095D1
:102F8000872F972F0E9428534B015C012DEB3EE1C8
:102F900040EC55E40E94AA5420E030E44CE955E4AA
:102FA0000E94F6510E94FA527B0121E33CE043E487
:102FB00055E4C501B4010E94AA5420E030E44CE17C
:102FC00056E40E94F6510E94FA521C9FF0011D9F88
:102FD000F00D1124E258FC4E86E0E192F192F38666
:102FE000E286778B668B8150C1F72196C830D10578
:102FF00019F6DF91CF911F91FF90EF90BF90AF90A6
:103000009F908F900895DF92EF92FF920F931F93FE
:10301000CF93DF93E82FD62E6BEA869F612D112484
:10302000669566956695F62FFF5F50E0683008F06C
:1030300071C0862F90E0880F991FEC01CC0FDD1F27
:10304000CC0FDD1FCC0FDD1FC80FD91FC40FD51F3C
:10305000CC0FDD1FC258DC4E0990D881C02DF8304E
:1030600008F47DC0DA01AA0FBB1FA658BB4E0D9114
:103070001C91DA01AA0FBB1FAA5ABB4E8D919C91DD
:103080009801281B390BAF2FB0E017970E94CD5144
:10309000600F711F811D911D6115710521E082076F
:1030A000910508F072C09BEAE99F912D1124969535
:1030B00096959695892F880F890F880F880FE81BA2
:1030C000F0E0EE0FFF1FEF5AFC4EE080F1808B0125
:1030D0000C1B1D0B8D2D90E0A0E0B0E06627782F33
:1030E000892F9A2F2CE030E040E050E00E94CE562D
:1030F0002E0D3F1D411D511DD8010E948356C80F42
:10310000D91FCE01DF91CF911F910F91FF90EF90CA
:10311000DF900895EA01CC0FDD1FC658DB4E099001
:10312000D881C02DDA01AA0FBB1FAA5ABB4E8D91C0
:103130009C919E01281B390BA62FB0E017970E9487
:10314000CD516C0F7D1F811D911D6115710521E011
:1031500082079105F8F4EB01F83008F083CF8F2F48
:1031600090E0880F991FDC01AA0FBB1FAA0FBB1F9D
:10317000AA0FBB1FA80FB91FA40FB51FAA0FBB1F13
:10318000A258BC4E6D917C918ECF6FEF7FEF80E0A7
:1031900090E089CF6FEF7FEF80E090E0EB01DCCF34
:1031A000EF92FF920F931F93CF93DF9380E0E82F6E
:1031B000F0E0EE0FFF1FEC53FD4E118210828F5F87
:1031C0008231A9F71092E9121092E8128091091346
:1031D000823009F44FC0833099F1813039F0DF91AA
:1031E000CF911F910F91FF90EF9008950091C2121F
:1031F0001091C312E0900813EE0CF12C4F2D60E0FB
:103200008E2D01DFEC014F2D60E080E0FCDE9E01A1
:10321000281B390BEF2DF0E0EE0FFF1FEC53FD4E96
:10322000D8010E94CD5191838083F3948CE0F812F1
:10323000E5CFDF91CF911F910F91FF90EF9008950F
:1032400020910813A091C212B091C31230E00E94E5
:10325000CD519B01AC01A5E5B5E10E948356909349
:10326000E9128093E812DF91CF911F910F91FF90A7
:10327000EF90089520910813A091C212B091C3124B
:1032800030E00E94CD519B01AC01A5E5B5E10E9463
:103290008356BB2797FDB095AB2F9093DD1280939B
:1032A000DC129093DF128093DE129093E1128093F0
:1032B000E0129093E3128093E2129093E5128093D0
:1032C000E4129093E7128093E612DF91CF911F9161
:1032D0000F91FF90EF90089520913C1030913D1098
:1032E0002F3F8FEF380791F080913A1090913B106B
:1032F000019690933B1080933A108217930730F019
:1033000010923B1010923A1081E0089580E00895E9
:103310000F931F93CF93DF93FC018BE1DF011D928D
:103320008A95E9F70EEC14E160E070E080E89FEB2D
:10333000C0E0D0E01BC0BE01882777FD8095982FA4
:103340000E94285320E030E04FE753E40E9461528E
:1033500020E030E040E85FE30E94F6512BED3FE0D3
:1033600049E450E40E94AA540E945E5220E030E0FA
:1033700040E85FE30E94F65120E030E040E05FE388
:103380000E94AA5420E03FEF4FE757E40E94AA545E
:103390000E94FA52F801619371938F012196C11531
:1033A000F1E0DF0741F6DF91CF911F910F91089572
:1033B00021E030E002C0220F331F8A95E2F7D901E5
:1033C000A095B0958091430A9091440A8A239B234B
:1033D0009093440A8093430AE091450AF091460A8B
:1033E000EA23FB23F093460AE093450A662371F033
:1033F000822B932B9093440A8093430A442331F009
:103400002E2B3F2B3093460A2093450A089524E63D
:1034100030E040E050E00E94A7562AE030E040E073
:1034200050E00E94A756605D205D30E020383105F5
:1034300088F4F901EC5AF94F80818093470A70E0D3
:103440006038710570F4FB01EC5AF94F808180936C
:10345000480A08958FEF8093470A70E0603871053D
:1034600090F38FEF8093480A089590E0803891059B
:1034700088F4FC01EC5AF94F80818093470A70E090
:103480006038710570F4FB01EC5AF94F808180932C
:10349000480A08958FEF8093470A70E060387105FD
:1034A00090F38FEF8093480A08951F93CF93DF9393
:1034B0001FB7F89453DD0E94133E109236101092FD
:1034C000351010921E1010921D10CFEFDFEFD09329
:1034D0001210C09311101092201010921F10D09350
:1034E0001410C09313101092221010922110D09338
:1034F0001610C09315101092241010922310D09320
:103500001810C09317101092261010922510D09307
:103510001A10C09319101092281010922710D093EF
:103520001C10C0931B10809139108160809339105A
:103530000E940C11D0932C10C0932B1010922E10BF
:1035400010922D10C0E06C2F6E5E8C2F0E94F73F02
:10355000CF5FC630C1F7809139108E7F80933910CC
:103560000E940C11809139108860809339100E945C
:103570000C1110922C1010922B108FEF9FEF909344
:103580002E1080932D106C2F645F8C2F0E94F73FBC
:10359000CF5FCC30C1F780913910877F809339108D
:1035A0000E940C1110922C1010922B1010922E10C1
:1035B00010922D108FEF9FEF90933610809335105F
:1035C00010921210109211101092141010921310E9
:1035D00010921610109215101092181010921710C9
:1035E00010921A101092191010921C1010921B10A9
:1035F0006C2F6A5F8C2F0E94F73FCF5FC231C1F7FB
:10360000109236101092351010921E1010921D104C
:103610001092201010921F10109222101092211060
:103620001092241010922310109226101092251040
:1036300010922810109227100E94863D1092470A7F
:103640001092480A1092440A1092430A1092460AB5
:103650001092450A10924D0A5AD01FBFDF91CF91A8
:103660001F9108958F929F92AF92BF92CF92DF9257
:10367000EF92FF920F93CF93DF93EC0180918C0F29
:1036800090918D0F8C589D4081309240A0F5862EF0
:10369000912C8114910479F181E0881A9108A12C70
:1036A000B12C2FEF821A920AA20AB20ABA2CA92CC4
:1036B000982C8824C12CD12C7601CE01A0E0B0E05A
:1036C000803E9105A105B10560F4A6014457524F13
:1036D0009F5FAF4FBF4F6627782F892F9A2F0E9489
:1036E00000F821968FEFD81AE80AF80AC814D9040E
:1036F000EA04FB0411F7DF91CF910F91FF90EF9057
:10370000DF90CF90BF90AF909F908F9008950F93D0
:103710001F93CF93DF931FB7F894F2DBC0918C0F08
:10372000D0918D0FAE0160E070E004E2069FF001E1
:10373000079FF00D1124E258FC4E80E090E02191AB
:103740003191DA01A80FB91F2D933C930296843270
:103750009105A9F76F5F7F4F4C5D5F4F6830710532
:1037600029F78091A0149091A114FE01E05EFE4F14
:1037700091838083FE01EE5DFE4F80919E149091B7
:103780009F1491838083CC5DDE4FD0938D0FC093C7
:103790008C0F8091A2148883E0918C0FF0918D0F93
:1037A000CF01019690938D0F80938C0F8091A3147D
:1037B0008183E0918C0FF0918D0FCF010196909352
:1037C0008D0F80938C0F8091A5148183E0918C0FD5
:1037D000F0918D0FCF01019690938D0F80938C0FF8
:1037E0008091A4148183E0918C0FF0918D0FCF0113
:1037F000019690938D0F80938C0F8091A6148183F6
:10380000E0918C0FF0918D0FCF01019690938D0F69
:1038100080938C0F8091A7148183E0918C0FF0919D
:103820008D0FCF01019690938D0F80938C0F809117
:10383000A8148183E0918C0FF0918D0F8091491332
:1038400090914A139093AA148093A9149283818330
:103850003396F0938D0FE0938C0F62E08CED90E047
:1038600001DF1FBFDF91CF911F910F910895CF927C
:10387000DF92EF92FF920F931F93CF93DF9300D0CD
:10388000CDB7DEB78091FF12182F110F180F1F5FF1
:103890008091FE12809350128091361290913712CF
:1038A000A0913812B0913912892B8A2B8B2B51F4AD
:1038B0006091870D7091880D8091890D90918A0D8E
:1038C0000E944B560E9448566093361270933712EE
:1038D000809338129093391280914E12181709F183
:1038E00010934E1286E392E10E944414A0914F126D
:1038F000BB27A1950CF4B095AA0FBB1F1196209180
:103900003E1230913F1240914012509141120E945C
:103910008D56609342127093431280934412909399
:1039200045128091ED129091EE12A091EF12B0919C
:10393000F0128F3F2FEF9207A207B20709F4B3C02E
:1039400020914113309142132115324008F074C088
:103950004FEF5FEFE090C012F090C11200900A1399
:1039600002C0F694E7940A94E2F78091391390919B
:103970003A13811562E0960708F4E7C09C013250C3
:1039800080914513909146139695879596958795C6
:103990008115E2E09E0708F489C08C0112508091E5
:1039A0000C13882309F488C0AA27249FB12D359FC2
:1039B000C001529FB00D811D9A1F349FB00D811D13
:1039C0009A1F112460913713709138138093461217
:1039D0009093471280914812909149126817790785
:1039E00021F086E392E10E946A14C80180959095C7
:1039F0008E159F0508F0ACC00FEF1FEF60914313C9
:103A000070914413109362120093611280916312BB
:103A1000909164126817790709F48CC081E592E1EE
:103A20000F900F90DF91CF911F910F91FF90EF902A
:103A3000DF90CF900C946A142091F1123091F21221
:103A400040E050E0820F931FA41FB51FC090870D68
:103A5000D090880DE090890DF0908A0DC816D90697
:103A6000EA06FB0600F1C090870DD090880DE0902B
:103A7000890DF0908A0DC81AD90AEA0AFB0AC21603
:103A8000D306E406F50608F063CF9E2D8D2D7C2D20
:103A900066270E94CE56F901EE0FFF1FE05EFC4F35
:103AA0004081518157CF40E050E054CF00E010E01A
:103AB00080910C13811178CFC901809590958E1556
:103AC0009F0508F048C02FEF3FEF609137137091CA
:103AD00038133093471220934612809148129091E8
:103AE00049126817790741F086E392E149835A83C6
:103AF0000E946A145A814981AA27049FB12D159FFB
:103B0000C001509FB00D811D9A1F149FB00D811DE3
:103B10009A1F112460914313709144138093611292
:103B200090936212809163129091641268177907E2
:103B300009F074CF0F900F90DF91CF911F910F91EB
:103B4000FF90EF90DF90CF90089520E030E018CF05
:103B50000E0D1F1D53CF2E0D3F1DB7CFAF92BF923D
:103B6000CF92DF92EF92FF920F931F93CF93DF9349
:103B700000D0CDB7DEB76C017B0180917D13811140
:103B800059C0042F017040FD48C0142F127041FD30
:103B90003CC021110DC00F900F90DF91CF911F916C
:103BA0000F91FF90EF90DF90CF90BF90AF9008956E
:103BB000002351F08091CF169091D0168C259D2531
:103BC0008C7F892B09F0F1C0112329F38091D11644
:103BD0009091D2168E259F2588279E7F892BD9F21A
:103BE0000F2D06954091A4144F70406BE0917B1906
:103BF000F0917C1921E063E070E08BE799E1099591
:103C0000F092D216E092D116C6CFF092C112E09295
:103C1000C0122A832CDE2A81BCCFD092C312C0925C
:103C2000C2122A834983BCDA6FEF81E0C9D7498188
:103C30002A81ABCF60E070E05FEFFB01EE0FFF1F6A
:103C4000E60FF71FEE0FFF1FEE0FFF1FEC56F44FAE
:103C500092859923F1F0852F992787FD9095DC01B6
:103C6000AA0FBB1FA80FB91FAA0FBB1FAA0FBB1F0C
:103C7000AC56B44F00811181228133818D919D9189
:103C80000D90BC91A02D80179107A207B30708F4EF
:103C9000562F6F5F7F4F6630710579F65F3F09F4ED
:103CA0007ACF852F992787FD9095FC01EE0FFF1F96
:103CB000E80FF91FEE0FFF1FEE0FFF1FE556F44F41
:103CC000808140FD68CF41FF66CF1BEA819F112DA7
:103CD0001124169516951695912F990F910F990FFE
:103CE000990F182F191BB70180E090E00E9426530E
:103CF00020E830E040E857E30E94AA546B017C01C1
:103D0000612F70E080E090E00E94265320E030E0D8
:103D100040E05FE30E94F5519B01AC01C701B60191
:103D20000E94F651D62EE72EF82E092F20E030E023
:103D3000A9010E945A5287FD55C020E030E040E4BE
:103D400051E46D2D7E2D8F2D902F0E943654181624
:103D50002CF4D12CE12C90E4F92E01E4A12EB12C0D
:103D6000AA0CBB1C81E593E1A80EB91E2BEA3AEA26
:103D70004AEA55E46D2D7E2D8F2D902F0E94AA5476
:103D80000E94FA52F501718360830ADA6FEF81E0D5
:103D90000F900F90DF91CF911F910F91FF90EF90B7
:103DA000DF90CF90BF90AF900BC7C60190589C0199
:103DB0003595279535952795092F06952F77332724
:103DC0004091A4144F70406EE0917B19F0917C19E2
:103DD00063E070E08BE799E10995D092D016C0922C
:103DE000CF16F2CED12CE12CF12C00E0B7CF809190
:103DF000A31487FD09C06F7070E0992787FD909527
:103E00006817790709F0089580E8289F9001112428
:103E1000242BC901905220E041E060E070E0880F5F
:103E2000991F880F991F9ACE4F925F926F927F923F
:103E30008F929F92AF92BF92CF92DF92EF92FF92BA
:103E40000F931F93CF93DF9380919E1490919F14B3
:103E50009093010180930001C0900401D09005016E
:103E60007C01EC18FD08C80ED91EC0910201D0914A
:103E7000030197012C1B3D0B40E050E0812C912C5D
:103E8000A12C60E8B62EC501B4010E94CE562901CE
:103E90003A012093060130930701409308015093A3
:103EA00009018E010095109598012C193D0940E0FB
:103EB00050E0C501B4010E94CE5649015A01209339
:103EC0000A0130930B0140930C0150930D01809136
:103ED000D30F9091D40F08171907B8F48FEF9FE70D
:103EE00020E041E060E070E0DF91CF911F910F9101
:103EF000FF90EF90DF90CF90BF90AF909F908F900A
:103F00007F906F905F904F9029CE8C179D07C0F0E7
:103F1000AC0160E070E08E159F0530F0C816D90640
:103F200090F080E090E0DCCFCB01BA016C1B7D0B00
:103F300081099109A30192010E94D3519058D0CFD9
:103F400080E090E8CDCF9A01AB012C193D094109E1
:103F50005109C501B4010E94D35190589058C0CF67
:103F6000CF93DF93CDB7DEB728970FB6F894DEBFB7
:103F70000FBECDBF92E09D8394E09E8397E09F8328
:103F80009CE0988795E0998393E09A8391E09B83E6
:103F90001C828230D9F1CCF0843009F461C06CF518
:103FA000DB01CA0181709927AA27BB2721E082275C
:103FB000809302134270552766277727759567957A
:103FC000579547954093031304C0882359F08130D7
:103FD00091F128960FB6F894DEBF0FBECDBFDF91EA
:103FE000CF910895440F551F661F771F8091FE12D1
:103FF0008170842B8093FE12ECCF853051F7FE0147
:10400000E40FF51F818180930A13E3CFDB01CA011E
:1040100081709927AA27BB2721E082278093041368
:104020004270552766277727759567955795479569
:1040300040930E13CECF809100138B7C41305105FD
:1040400061057105E1F04230510561057105E9F046
:104050004330510561057105B1F080930013B9CF6C
:10406000FE01E40FF51F85818093081328960FB693
:10407000F894DEBF0FBECDBFDF91CF91D5CE80616A
:1040800080930013A6CF8460E8CF806280930013F2
:10409000A0CF2F923F924F925F926F927F928F921A
:1040A0009F92AF92BF92CF92DF92EF92FF920F93C7
:1040B0001F93CF93DF93CDB7DEB760970FB6F89419
:1040C000DEBF0FBECDBF80902D1390902E139C8627
:1040D0008B86A0902513B0902613BE86AD86212C2A
:1040E000312CF3C083E0EF85F88980A7CF010E94CF
:1040F000CB3490910313992309F40CC183E0ED8133
:10410000FE8180A7CF010E94CB349091A714992300
:1041100009F4FCC01595812F992787FD909501968C
:1041200020FEFAC04FEF5FEF849F9001859F300D16
:10413000949F300D1124922F8827AC01662757FDDC
:104140006095762F80913113909132134A015B0173
:10415000880E991EA11CB11CD501C401B7FCF5C085
:1041600020912F13309130136A017B01C20ED31EB0
:10417000E11CF11CF7FCE5C020912B1330912C13AE
:104180004A015B01820E931EA11CB11C89829A8296
:10419000AB82BC82B7FCD0C02091291330912A1386
:1041A0004A015B01820E931EA11CB11CB7FCC0C06A
:1041B00020912713309128132A013B01420E531EF0
:1041C000611C711C77FCB0C0009123131091241363
:1041D000F8018A019B010E0F1F1F211D311D0F8346
:1041E000188729873A8737FD9AC009811A812B8160
:1041F0003C8101151105F1E02F07310524F00FEF87
:104200001FEF20E030E0C982DA82EB82FC82C11429
:10421000D10441E0E406F10444F04FEF5FEF60E0C9
:1042200070E049835A836B837C83BC01CD016115A7
:10423000710551E08507910524F06FEF7FEF80E075
:1042400090E09FE0C92EE12CF12C2B853C85498123
:104250005A818F8598890E94C0350F8118852985DC
:104260003A850115110561E02607310524F00FEFAD
:104270001FEF20E030E0B301A2014114510481E0BE
:104280006806710424F04FEF5FEF60E070E0811486
:10429000910491E0A906B1042CF088248A94982C0A
:1042A000A12CB12CBFE0CB2EE12CF12C2D853E852D
:1042B000B4018D819E810E94C035EFEF2E1A3E0A17
:1042C000F6E02F16310409F444C0122D5AE2B52E3F
:1042D000B29CC001B39C900D11249C01265C3E4E03
:1042E000388B2F8720910413EF85F88926A39C0132
:1042F000225C3F4E3E832D8390910213F90196A3D9
:1043000090910E139111EECE81E0EDCE40E050E0A1
:10431000BA0118CF81E0F3CE41E050E005CF1F8213
:10432000188619861A8661CF412C512C32014CCF48
:10433000812C912C54013CCF19821A821B821C8241
:104340002BCFC12CD12C760117CF80E090E0DC017F
:1043500007CF60960FB6F894DEBF0FBECDBFDF91DA
:10436000CF911F910F91FF90EF90DF90CF90BF9072
:10437000AF909F908F907F906F905F904F903F9005
:104380002F900895CF92DF92FF920F931F93CF93B8
:10439000DF931F92CDB7DEB781E00E94ED130E943C
:1043A0007E348091061381114DC00E940642109107
:1043B000A5148091E30B181721F081E04ED21093E1
:1043C000E30B109107138091E20B181731F081E095
:1043D00044D21330A8F51093E20B49DA5ADE0E945A
:1043E000D018F090A81464EBC62E62E1D62E2CE013
:1043F0000FEF1FEF09C0F601118300832F5FF2E07A
:10440000CF0ED11C223191F0FF20A9F3422F60E0A2
:104410008EE729830E940318F60191838083298106
:104420002F5FF2E0CF0ED11C223171F70F90DF9198
:10443000CF911F910F91FF90DF90CF900C94A431FA
:1044400010E0C9CF61E08BE493E12BD2B0CFCF93E2
:10445000DF932091A31427FD0BC06F7070E033270A
:1044600027FD30956217730719F0DF91CF910895FA
:104470008091A2148823C9F34436B8F7C42FD0E042
:104480008091A0149091A114C817D90771F3CE019F
:104490000E94DD16882349F3D093A114C093A01481
:1044A00010926B1334D9DF91CF916CCFE82FF0E0ED
:1044B000ED53F64F90819170803209F456C078F038
:1044C000843209F44CC0A0F1863209F445C008F0EA
:1044D00058C09093FC1281E080936B1353CF8C31C2
:1044E000C8F08C3109F444C08091E009817090914A
:1044F00000139473892B9091E10990FD47C090E0DF
:10450000892B9091E20990FF45C092E0892B80931E
:104510000013E1CF8A31A8F08091DE09817090917B
:10452000DD0990FD35C090E0892B80930113D3CF36
:104530008232C1F018F09093F812CDCF9093F6121A
:10454000CACF883131F0893109F008959093FA1279
:10455000C2CF9093F712BFCF9093FD12BCCF909330
:10456000F912B9CF9093FB12B6CF9093F512B3CF57
:104570009091DF098091FE1290FB80F98093FE12EA
:10458000AACF873211F790930613A5CF98E0B8CF42
:1045900092E0CACF90E0BACFCF938091A214882343
:1045A000D1F08091A0149091A1140E94DD1688236F
:1045B000C1F08091A2148823D9F00E94A813109210
:1045C0006B1381E09091A214911101C080E080935F
:1045D0006913CF9108958BED90E00E94DD16811153
:1045E000E8CF81E00E9496158091A2148111E5CF59
:1045F000C8E18C2F5BDFCF5FC832D9F781E00E9422
:104600009240DBCFCF93DF93C42FD22F8091A3149E
:1046100087FD0BC06F7070E0992787FD9095681734
:10462000790719F0DF91CF910895C11135C020911C
:10463000A214D23008F481C02223A1F38C2F805120
:104640008E3198F18C2F80558E3108F04FC0EC2FB1
:10465000F0E0EE0FFF1FE159FD4E408151812D2FFB
:1046600030E0CA0196958795969587958F7799271B
:1046700082179307B9F2CA0188279E7F220F331F42
:10468000220F331F822B932B9183808381E08093B1
:104690006B13DF91CF9176CEC13009F461C0C03485
:1046A00009F469C02091A214C7CFEC2FF0E0EE0FFF
:1046B000FF1FE151FD4E808191812D2F30E0AC0133
:1046C000452F552746954217530709F4ABCF8C7FEA
:1046D0009170322F2227330F822B932B918380836B
:1046E00081E080936B13DF91CF914CCE8C2F805360
:1046F0008A3108F097CFEC2FF0E0F0972D2F30E0C3
:10470000DF01AC52B94F4C9187E090E0841B9109D6
:1047100002C0359527958A95E2F7822FDF01AB50CD
:10472000BD4E9C91291709F43EC02C93C1E07197AE
:1047300061F1CC2309F476CFA9CF622F772767FDEB
:1047400070958D2F90E06817790709F475CFD09395
:10475000A2140E94871B20DF15DE2091A2146CCFCB
:104760007D2F770F20E042E060E080E090E0F6D916
:104770002091A21461CFD11104C0DF91CF910C948C
:10478000883681E08093E50B4DCF882371F00E943D
:10479000244286E0ECEDFBE0ABE4B3E101900D9246
:1047A0008A95E1F7C6CFC0E0C2CF0E940642F1CFA2
:1047B0008091A614813009F008956A3FB1F06C3FF2
:1047C00041F0683FC9F78091F3128F5F8093F31235
:1047D00008958091E60B823089F180916E0C8230D1
:1047E00059F78EE69CE00C94F43A8091E60B823007
:1047F00079F11092690C1092680C8FEF9FEF9093F3
:104800006B0C80936A0C80916E0C8230E1F01092F8
:10481000F10C1092F00C8FEF9FEF9093F30C8093BC
:10482000F20C90937A0D8093790D8FEF9FE7909320
:104830003B1080933A101092F312089586EE9BE09D
:104840000E94F43ACACF8EE69CE00E94F43ADFCF91
:1048500086EE9BE00E94F43ACCCFEEE9FBE09FEFBE
:10486000DF0112971C921082DF0113979C93DF01E6
:1048700014979C93DF011A971D921D921D921C9212
:1048800013973C962BE0E63EF20751F7811101C0E9
:10489000089580E1E4E8FAE0DF011D928A95E9F7E6
:1048A00008951F93CF93DF93182FD92FC62F809190
:1048B000E40B8617F1F080E0D0DFC093E40B46E014
:1048C00050E06FEF70E08CED9BE00E94E455E12F2B
:1048D000FD2FACEDBBE080E091919F3FB9F09D933F
:1048E0008F5F8630C9F71092DC0BDF91CF911F915B
:1048F000089546E050E06CED7BE0812F0E94BD55AD
:104900000097D9F6DF91CF911F9108958111EBCFD8
:10491000ECEDFBE086E0DF011D928A95E9F7DF917F
:10492000CF911F910895CF93DF93FC01D62FCFB77E
:10493000F894218130E0C90101964281642F70E032
:104940000E94E251408150E08417950791F0A381C5
:10495000B481A20FB31FDC93818190E00196628144
:1049600070E00E94E2518183CFBF81E0DF91CF915F
:104970000895CFBF80E0DF91CF910895FC013FB74C
:10498000F89421819081291728F48281820F891B54
:104990003FBF0895822F891B3FBF0895AF92BF92FA
:1049A000CF92DF92EF92FF920F931F93CF93DF93FB
:1049B000082FD62EC0E0D0E088E8E82E98EEC92E69
:1049C000C00E2FE3F22E1FEFEC9EF001ED9EF00DD6
:1049D0001124EA51F44F8081833079F02196C2305E
:1049E000D10591F7DF91CF911F910F91FF90EF903B
:1049F000DF90CF90BF90AF9008950C3F09F45AC05C
:104A00000D3F09F46AC00E3F09F48CC0DD2091F11E
:104A10004091F80C842F8F5F8093F80C5F0161E860
:104A2000A60EB11CD5016C91862F90E02091F70C59
:104A3000DC01A20FB11DA038B10584F6442309F4AE
:104A40009EC0462F4150242F332727FD30952E5FDF
:104A50003F4F2E0F3F1FD9015E919D01752F7F7330
:104A6000C71609F4BBCF57FF03C0415047FFF3CF30
:104A700020E88DC08091F80C811177C05F0161E85A
:104A8000A60EB11CD5012C9130E02F5F3F4F2E0FA9
:104A90003F1F4091F70C50E06EE370E0C9010E94A7
:104AA000E4558091F70CF5019081890F8083109275
:104AB000F70C94CFDF01AF57BF4F1C92DF01AA570D
:104AC000BF4F1C921092F70C319640E850E06FEF08
:104AD00070E0CF010E94E45581CFDF01AA57BF4F9C
:104AE0008C91882309F47ACF81508C938091F70CB4
:104AF000811141C05F0161E8A60EB11CD5018C9106
:104B0000882309F46BCF8150D5018C939F01280F26
:104B1000311DD90111969C91119711961C9397FF05
:104B20005DCFEECF5F01B1E8AB0EB11CD5014C916A
:104B3000842F90E02091F70CBC01620F711D60384A
:104B400071050CF04BCF9F012A573F4FD9015C9163
:104B50005F5F5C932091F80C211122C0E80FF91FD0
:104B6000F1824F5FF501408339CF81508093F80C7B
:104B7000811134CF83CF81508093F70C2FCF9F01C9
:104B80002A573F4FD9014C914F5F4C9320E0E80FDB
:104B9000F91F822F8C2981836F5FF50160831ECFFF
:104BA0008091F70C8F5F8093F70C18CF211106C00E
:104BB000472F582F692F7727CA0108950C94961410
:104BC0002F923F924F925F926F927F928F929F921D
:104BD000AF92BF92CF92DF92EF92FF920F931F930B
:104BE000CF93DF93CDB7DEB7A0970FB6F894DEBFB3
:104BF0000FBECDBF8C87362E882309F49BC0E09171
:104C00001B13F0911C1340901D1350901E134091E4
:104C10000F1350911013809115139091161320913A
:104C20004713309148130091D10F1091D20F20906B
:104C3000011360910B131093D4160093D316F093C5
:104C4000D616E093D5165092D8164092D7165093A8
:104C5000DA164093D9169093DC168093DB163093C6
:104C6000DE162093DD162092DF166093E016000F0B
:104C7000012F001F110B11951A95EE0FEF2FEE1F4C
:104C8000FF0BF1955F01BA94612C712C73016201E5
:104C9000CC0CDD1CEE1CFF1CCC0CDD1CEE1CFF1C28
:104CA000C40CD51CE61CF71C73E0F694E794D7946B
:104CB000C7947A95D1F756954795569547954C01E7
:104CC00096948794969487948D2D99279B878A87AD
:104CD000A52FBB27BF83AE83E92DFF27F987E88780
:104CE000D701C6019927AA27BB278B8B9C8BAD8B3D
:104CF000BE8B662309F443C0623008F430C29CE0E6
:104D0000E92EF12C8E819F81B7010E94E251AE8184
:104D1000BF81A81BB90BBF83AE83CF01B7010E942F
:104D2000E251E81BF90BF987E887188A1F861E866F
:104D30001D862DC00091D10F1091D20F8091D316F6
:104D40009091D416E0911B13F0911C1380179107DA
:104D500009F4E1C140901D1350901E1340910F13B0
:104D600050911013809115139091161320914713B1
:104D7000309148132090011360910B135CCFFA011E
:104D8000FF27FE87ED87A4015527588B4F87509149
:104D90000613598B7091A7147D8F832F99279C8FB1
:104DA0008B8F3091EC123A8BE12CF12C58E15D8322
:104DB00020E0B801882777FD8095982F69837A8352
:104DC0008B839C83C501AA2797FDA095BA2F8F8B53
:104DD000988FA98FBA8FF8A2EF8E0AC02F5F4F8DE0
:104DE00058A14E5F5F4F58A34F8F263009F438C14A
:104DF00037FC02C02311F2CF8F8D98A1880F991F25
:104E0000AF8CB8A08A0D9B1D880F991F8C57954FAA
:104E1000FC01E85EFE4F3081332309F43AC1FC0106
:104E2000E95EFE4FB080BD823D81A32EB12C48E1EA
:104E3000A41AB108888499848A0C9B1C0F8D18A130
:104E4000025C1F4EF801EA57FD4FC080D180EE246E
:104E5000D7FCE094FE2C69817A818B819C81C60EFF
:104E6000D71EE81EF91E8E819F818A0D9B1D97FD1E
:104E700027C1422F6D852E8F0E940318C80ED91EA0
:104E8000E11CF11C2E8DF7FC29C1C114D10471E085
:104E9000E706F1042CF0CC24CA94DC2CE12CF12C94
:104EA000F801EE56FD4F40805180662457FC609417
:104EB000762C89819A81AB81BC81480E591E6A1E6D
:104EC0007B1E4F89588D698D7A8D440E551E661E46
:104ED000771E422F4A5FC40197FCFDC06F852E8F5D
:104EE0000E940318480E591E611C711C2E8D77FC00
:104EF000EEC04114510451E0650671042CF04424C5
:104F00004A94542C612C712C8A859B85222051F067
:104F100061E0261609F4F2C08A859B858A0D9B1DE7
:104F200097FDF6C0422F445F6B892E8F0E940318B5
:104F3000F801E256FD4F80809180AA2497FCA0944E
:104F4000BA2C880E991EA11CB11C2E8DB7FCBBC0BB
:104F50008114910481E0A806B1042CF088248A947D
:104F6000982CA12CB12C3989311104C05D8D5523A9
:104F700009F451C0822F8595992787FD9095019658
:104F800020FF9BC06FEF7FEF869FA001879F500D92
:104F9000969F500D11246B8D7C8D469FC001479FBD
:104FA000900D569F900D1124AA2797FDA095BA2F1A
:104FB000C80ED91EEA1EFB1EF7FC9CC0C114D1040A
:104FC00071E0E706F1042CF0CC24CA94DC2CE12C2F
:104FD000F12C480E591E6A1E7B1E77FC87C04114B7
:104FE0005104E1E06E0671042CF044244A94542CE0
:104FF000612C712C880E991EAA1EBB1EB7FC72C0B4
:1050000081149104F1E0AF06B1042CF088248A9455
:10501000982CA12CB12CAA88F801AA2009F43EC032
:10502000EE5AFD4FD182C082F801E25AFD4F518203
:105030004082F801E659FD4F918280822110CECE48
:10504000F801EA5BFD4F91828082C8CE6091DF1645
:105050002612B7C060910B137091E0166713EBCD69
:10506000A0960FB6F894DEBF0FBECDBFDF91CF91F3
:105070001F910F91FF90EF90DF90CF90BF90AF9076
:105080009F908F907F906F905F904F903F902F9068
:1050900008953C853F3F09F0A1CEC6CEE25DFD4FAD
:1050A000D182C082F801E65CFD4F51824082F80156
:1050B000EA5BFD4F9182808291CE61E070E064CF27
:1050C00080E090E0D6CE812C912C540141CF412C30
:1050D000512C32010ECF80E090E000CFC12CD12CBA
:1050E0007601D3CE812C912C54018ACF412C512CA6
:1050F000320175CFC12CD12C760160CFB7FC34C002
:10510000B594A7948A859B858A0D9B1D97FF0ACF2E
:1051100080E090E007CF8091D5169091D616409010
:105120001D1350901E13E817F90709F017CE809150
:10513000D7169091D81640910F135091101348161E
:105140005906B1F0809115139091161320914713D1
:10515000309148132090011360910B136CCD188A85
:105160001F861E861D8613CE7FEFA71AB70AC8CFEB
:105170008091D9169091DA164817590719F780913E
:105180001513909116132091DB163091DC168217BF
:10519000930749F020914713309148132090011351
:1051A00060910B1348CD20914713309148136091C3
:1051B000DD167091DE16209001132617370709F4CB
:1051C00045CF60910B1337CDCF92DF92EF92FF92D4
:1051D000CF939091F7122091FA12992309F492C07B
:1051E000409113135091141360E070E0222309F4EE
:1051F00085C0C0901913D0901A13E12CF12C88238C
:10520000A1F0992381F08091001385FD0CC080915D
:105210004C1290914D12AA2797FDA095BA2F480FD6
:10522000591F6A1F7B1F211172C0CFB7F894411517
:10523000510521E06207710524F04FEF5FEF60E058
:1052400070E0DB01CA0177FD77C00E94940E46EC46
:1052500041BB469A31E035B921E428B950EF5BB93A
:1052600092EA9EB987E881BB00C000C041BB469A64
:1052700035B928B960E76BB99EB981BB00C000C0E1
:1052800041BB469A35B928B95BB99EB981BBD701F4
:10529000C601C114D10421E0E206F10424F08FEF2D
:1052A0009FEFA0E0B0E0B7FD43C00E94940E46EC33
:1052B00041BB469A31E035B927E428B950EF5BB9D4
:1052C00092EA9EB987E881BB00C000C041BB469A04
:1052D00035B928B960E76BB99EB981BB00C000C081
:1052E00041BB469A35B928B95BB99EB981BBCFBFDE
:1052F000CF91FF90EF90DF90CF900895C12CD12CEB
:1053000076017DCF4FEF5FEF60E070E06FCF80916F
:10531000001384FD8ACF80914C1290914D12AA27E0
:1053200097FDA095BA2FC80ED91EEA1EFB1E7DCF91
:1053300080E090E0DC01B9CF80E090E0DC0185CF37
:1053400086EC81BB469A15B896E898B993E09BB96C
:105350001EB897E891BBEFE9FFE03197F1F700C085
:10536000000081BB469A15B823E828B923E12BB980
:1053700022E02EB991BBFAE0FA95F1F700C081BBAB
:10538000469A20EE27B997E09AB92DB915B820E8CA
:1053900028B99BB91EB897E491BB92E09A95F1F7B2
:1053A00000C096B199B19CB181BB479A87EE87B98D
:1053B00087EF8AB982EE8DB9EAE0EA95F1F700C08D
:1053C00008951F93CF93DF93D82FD86F8695869536
:1053D000869528E030E001C0220F8A95EAF7C22FB7
:1053E000C095CD231FB7F894CB010E94940EE6EC34
:1053F000E1BB469A3D2F330F367031649D2F969551
:105400009270906A71E075B938B9A0EFABB99EB9E6
:1054100067E861BB85E08A95F1F70000E1BB469A39
:10542000FC2FFF0F4C2F46955C2F551F5527551FFE
:105430008F2F8670582B5064C0718F2F880F807209
:105440008C2BF07C8F2B4270406A75B958B98BB9A0
:105450004EB961BB8AE08A95F1F700C0E1BB469A7C
:1054600075B938B9ABB99EB961BB8AE08A95F1F7D5
:1054700000C01FBFDF91CF911F9108952F923F92DF
:105480004F925F926F927F929F92AF92BF92CF9214
:10549000DF92EF92FF920F931F93CF93DF93CDB7DD
:1054A000DEB7CD55D1090FB6F894DEBF0FBECDBF24
:1054B000882309F408C3512C352C330C330C330CDE
:1054C000E6EC4E2ECC24C394D12CCC0EDD1E9E01D6
:1054D000255F3F4F69963FAF2EAF69974FB7F8945E
:1054E00041BA469A952D990F292F26702064892F4D
:1054F000880F8072907C892B952D9695927031E063
:1055000035B928B98BB99EB987E881BB5DE05A955A
:10551000F1F7000041BA469A80EE87B997E09AB950
:105520008DB935B980E488B91BB88EB987E481BBE1
:1055300062E06A95F1F700C026B199B18CB141BA29
:10554000479A622E669473E06722A0E82A9F900132
:105550001124622A292F2071622A292F2695269547
:105560002870622A96959076692A90E0880F991F94
:1055700084709927682A87EE87B987EF8AB982EE07
:105580008DB94FBF732C912C66E0262E7FE7A72E96
:10559000B12C09C08250808366949394739488E000
:1055A000981609F4D0C0072D10E0F801ED53F64F1E
:1055B0008081982F9E7F71F7962D9170817098173A
:1055C00059F3892F8A608083BFE3B71508F473C04D
:1055D000E92EFF24E7FCF094872D6E969FAF6E971F
:1055E0000E9456226E969FAD6E97E114F10409F465
:1055F000C9C0872D8051823008F4F4C1FAE07F16CB
:1056000009F4DFC13BE080917F0D731609F411C2EC
:10561000882309F4B7C05DE07512F6C061E090918F
:105620007E0D911160E00E94383991E0EF2809F475
:10563000B8C08091D20980FF14C1A9E0A71508F075
:1056400076C1B2E17B1609F404C6ECE07E1609F4DB
:1056500058C1FDE07F1609F416C290916913953088
:1056600009F419C1992309F431C279E0771508F4D6
:1056700098C0923009F47FC308F4DDC2953008F079
:1056800090C080916A13B72DAAE08A9FB00D1124B3
:105690008B2FB0936A13943009F452C5992787FD74
:1056A00090950E94DD1681112DC4EFEFE0936A13EF
:1056B0000E94CC2276C0492F552747FD50958091F6
:1056C0007813811171C08091791381116DC0452BC0
:1056D00051F08091E60B813009F4CFC280916E0CBD
:1056E000813009F4BFC240917F0D4111EBC0172DED
:1056F00018528091E60B833009F457C180916E0CEB
:10570000833009F452C18091F41221E040E050E866
:10571000692F810F6E969FAF6E970E94D036809151
:10572000F412810F6E969FAD6E979111BAC140E44D
:10573000682F8091A4140E948E126694939473949F
:1057400088E0981230CF5394380E9FE0951508F0FA
:10575000C5CEC35ADF4F0FB6F894DEBF0FBECDBF24
:10576000DF91CF911F910F91FF90EF90DF90CF903D
:10577000BF90AF909F907F906F905F904F903F90C1
:105780002F90089567E2761609F454C0E114F104ED
:10579000F1F53FE0731609F447C090E0EF2809F0F7
:1057A00048CF0E94C221F8CE452B09F4F5CEEEEE8B
:1057B000F6E0D6018AE001900D928A95E1F76996AC
:1057C000AEADBFAD6997E22D1D92EA95E9F7872D41
:1057D00088558093F4128093F60C80937C0D4AE0F8
:1057E00050E0BE01665F7F4F992787FD90950E942C
:1057F0005456C6010E94821380917813882309F4BD
:10580000CBCE10927913C8CE27E27216B1F07EE0AB
:10581000771681F15FE07512C0CF809179138823EC
:1058200009F4B3C010927913909378138FEF80939B
:105830007B13B3CFE114F104D1F00E942442ECEDCC
:10584000FBE0ABE4B3E1822D01900D928A95E1F784
:105850008091A2148111A1CF8BED90E00E94E943C9
:105860009CCFB2E17B12F1CE0E94551A9ACF0E94D2
:105870000642E5CF8091A214882309F4EECE8091F0
:105880006913882309F412C1109269139091691366
:10589000953009F0E7CE8091E60B833029F08091B6
:1058A0006E0C833009F07DCF32E0371508F479CFE4
:1058B000F801E05EF84F80818F3F09F472CF61E01C
:1058C0006DD86FCF272D20549111BEC080917E0DD1
:1058D000882309F48FC1413009F420C3E9EFFCE0CB
:1058E00080E090E005C001968038910509F454CE1F
:1058F00041912413F8CFFC01E750F34F2068208337
:105900004BCE8091A214811106C08BED90E00E94D5
:10591000E9438091A21491E0811190E09093A21448
:105920000E94871B0E94CC220E94C2213ACF109273
:105930007A131092791382E2EEEFF6E0DE01D3964D
:1059400001900D928A95E1F780917B13871509F4F8
:1059500018C270927B1384E0781609F49DC38715F2
:1059600008F072C1E8E07E1609F4EAC1E71508F410
:10597000BAC2F5E07F1609F474C326E0721211CFA3
:105980008CE099E00E9482130CCF80917A138823D7
:1059900009F490C010927A1381E080937913909368
:1059A00078138FEF80937B13F8CE692F812F6E963B
:1059B0009FAF6E970E94CE24C7D46E969FAD6E9710
:1059C000A2CE81E020917F0D213009F449C1609180
:1059D0007E0D6E969FAF6E970E9438396E969FAD82
:1059E0006E97D4CE81E0E1E17E1280E028E8829FCC
:1059F000F0011124EA51F44F2081213081F008F4A4
:105A0000EDC0223009F45DC1233009F0FBCD21E067
:105A10004091A214442309F463C12093691362E006
:105A20006E969FAF6E970E9472426E969FAD6E9774
:105A3000E5CD823009F42DC108F4C4C0833009F4E7
:105A400034C18111AACEA2CEA9EFBCE0FD0105C0F0
:105A50003DE0E937F30709F4FCC181918F3FC1F3C1
:105A6000413009F430C180E090E005C001968038F3
:105A7000910509F491CD4D914F3FC1F7FC01E750DD
:105A8000F34F208389CD9111E8CD80916913823045
:105A900009F465C1843009F462C182E0809369131E
:105AA00080CE60E070E80E94751276CD81E0809330
:105AB0006913D3CD8FE380937A13909378138FEF8C
:105AC00080937B136ACEA8E05A2EF6CC60917713B0
:105AD00059E0571508F465CE272D671509F404C160
:105AE000462F552747FD5095872D992787FD90957F
:105AF0000A964817590709F44DC2709277138FEF31
:105B00009FEFDC018093731390937413A09375132C
:105B1000B0937613822F992787FD90958C01000F03
:105B2000111F080F191F000F111F000F111F005E1A
:105B30001A4F0E94A813D80112966D917C91139769
:105B4000C6010E94F655F60101900020E9F7319751
:105B5000CF018C199D092DE330E240E02083318391
:105B60004283F8012081213009F48EC108F031C14F
:105B7000E2E0F0E0EC0FFD1FE80FF91F1082D80102
:105B80001196EC91EE0FFF0BE15FFC4E808191814D
:105B90009093721380937113A0E0B0E080936D1323
:105BA00090936E13A0936F13B0937013C6010E946D
:105BB00082138091A2148111F4CD8BED90E00E94AC
:105BC000E943EFCD60917E0D83E06E969FAF6E97B7
:105BD0000E9438396E969FAD6E97D8CD209169138B
:105BE000223009F46BC220917813222309F417CFD5
:105BF00061E016CF413009F45CC1E9EFFCE080E0E0
:105C000090E004C001968038910541F04191241341
:105C1000F9CFFC01E750F34F5FEF5083E9EFFCE071
:105C200081918F3F09F0B8CC7DE0E937F707C1F7E4
:105C30000E941C39B1CC913009F0B3CD70926A1337
:105C400083E080936913ADCD91E0791609F45BC0D0
:105C5000791608F03CC189E599E00E948213A1CD34
:105C600080E0B5CE62E06E969FAF6E970E94724262
:105C70006BD36E969FAD6E9736CD62E080E06E96E8
:105C80009FAF6E970E9472425FD36E969FAD6E97E4
:105C900025CD60917E0D80E06E969FAF6E970E943D
:105CA00038396E969FAD6E9771CD60917E0D82E012
:105CB0006E969FAF6E970E9438396E969FAD6E9725
:105CC00065CD60E0ADCE822F90E0FC01E750F34F50
:105CD0002083F501E81BF90BE750F34F20835CCCE0
:105CE00020E0209369139BCE265F209377138FEFDC
:105CF0009FEFDC018093731390937413A09375133B
:105D0000B093761307CF8091A314F60162E0860268
:105D1000E00DF11D112464A975A9C6010E94F65574
:105D2000D6010D900020E9F71197EEECF8E0822DF6
:105D300001900D928A95E1F7C6010E94821331CD40
:105D40008091A614813009F4F6C1823009F47AC238
:105D5000811127CD88E299E00E94821322CD81E053
:105D60009091A214911101C080E0809369132FEFEC
:105D700020936A1316CD70926A1384E0809369139E
:105D800010CDE4E07E1609F450C2E71508F4D7C040
:105D9000F1E07F1609F42AC27F1608F4BFC122E0A1
:105DA000721609F433C233E07312D3CD8091D30F4E
:105DB0009091D40F90939F1480939E140E94871B00
:105DC0000E94141F8DEA98E00E94821370927B1348
:105DD000E8CC223009F0EACE8AE1E5EFF2E1A1EE6B
:105DE000B6E101900D928A95E1F76D961CAE1DAE5D
:105DF0001EAE1FAE6D976A96FFAC6A976D964CAD5E
:105E00005DAD6EAD7FAD6D97F80181810E94B01FD1
:105E10004AE150E065EF72E181EE96E10E94BD55E6
:105E2000009709F49EC16D966CAD7DAD8EAD9FADB2
:105E30006D976F5F7F4F8F4F9F4F6D966CAF7DAFAC
:105E40008EAF9FAF6D97643071058105910599F60E
:105E5000ADCE8091A614EFEFFFEFF0937A0DE093B3
:105E6000790D8111FDCD8091E60B823009F4F8CDDA
:105E700080916E0C823009F4F3CD8FEF9FE7909301
:105E80003B1080933A10ECCDE181FF27E7FDF095C0
:105E9000EB50FD4EE081F0E03296EE0FFF1FE00F79
:105EA000F11F6081718102968C0D9D1D0E94F65537
:105EB0007DCE822F90E0FC01E750F34F6FEF6083BF
:105EC000F501E81BF90BE750F34F6083A7CEA2E082
:105ED0007A1609F4A9C0B3E07B1263CC8AED98E08E
:105EE0000E9482135ECC39E0731609F465C052E15A
:105EF000751257CC81E090917D139111DDC0809394
:105F00007D134FCC80916A13992787FD90959093CC
:105F1000A1148093A0140E94871BC7CB822F90E00E
:105F2000FC01E750F34F208120682083F501E81B36
:105F3000F90BE750F34F8081806880832DCB56E0CA
:105F4000751609F41BC1751608F4D5C068E07616FD
:105F500009F43BC179E07712FCCC81E09091A71461
:105F6000911101C080E09091A814911170C190E04E
:105F7000890F90E00196AC01417055274093A7141A
:105F80008370992786958093A8140E94871B0E948E
:105F9000C221DFCC262F2A50209377138FEF9FEF5B
:105FA000DC018093731390937413A0937513B093D3
:105FB00076136213AFCDF5CB88E0E5E4F9E0D601C6
:105FC00001900D928A95E1F78091A714811183C009
:105FD0008FE696E6A6E6B0E088879987AA87BB8712
:105FE000D6010D900020E9F7CD0101978C199D098C
:105FF000D601A80FB91F2CE0EDE4F9E001900D9255
:106000002A95E1F72091A814F601E80FF91F222341
:1060100009F49EC08FE69EE6A0E083879487A5875B
:10602000C6010E948213BDCB8091A414F60172E0D8
:106030008702E00DF11D112464A975A9C6010E9413
:10604000F655D6010D900020E9F71197E4EDF8E040
:10605000822D01900D928A95E1F7C6010E9482136C
:10606000A0CB20917C138091A51490E0022E02C059
:10607000959587950A94E2F780FD34C088E0E4E0C6
:10608000F9E0D60101900D928A95E1F72F5C2B8300
:10609000C6010E94821385CB86E593E6ADE2B0E0AF
:1060A00089839A83AB83BC8380917C138F5C8B83C1
:1060B000C6010E94821375CB80E021CF63E06E960B
:1060C0009FAF6E970E94724285E0809369136E962F
:1060D0009FAD6E9793CA8FE69EE6A0E0888799876A
:1060E000AA877ECF87E0EDEFF8E0D60101900D9210
:1060F0008A95E1F7CBCF81E090E000907C1302C05D
:10610000880F991F0A94E2F79091A514982790930D
:10611000A5140E94871B0E94C2211BCC81E00E9413
:10612000961581E080936B1389E699E00E948213B3
:106130000E94C2214BCE81E399E00E94821331CBB1
:10614000992787FD90950E94E94380916A13A6CA1A
:106150008FE696E6A6E6B0E083879487A587B687A4
:106160005FCFF8012F2D32E02302E00DF11D112445
:1061700064817581C6010E94EB5518CD67961FAEEC
:106180001EAE679700E010E005C00F5F1F4F04369A
:10619000110591F0C8010E94DD168823B1F3BE01FC
:1061A0006B5A7F4FC8010E94A41667968EAD9FADB3
:1061B00067970E949A41E9CF8FEB98E00E94821383
:1061C0000E94CC220E94C22101CE8091A614992760
:1061D00087FD9095019663E070E00E94E251809304
:1061E000A6140E94871B0E94C221B3CB8091A314E6
:1061F000992787FD9095029661E170E00E94E25137
:1062000081508093A3140E94871BA3CB8091A41478
:10621000992787FD909501968F70907897FD27C0FC
:106220008093A4140E94871B94CB80917C139927A0
:1062300087FD9095019666E070E00E94E2518093A0
:106240007C1387CB8BE399E00E948213AACA92E069
:106250008FCE10927A131092791382E2EEEFF6E06D
:10626000DE01D39601900D928A95E1F772CB0197EA
:10627000806F9F6F0196D4CF0F931F93CF93DF93BF
:106280008091D30F9091D40FE0910001F091010122
:10629000A0910401B0910501609102017091030188
:1062A0009B01209530952817390740F42FEF3FE7E1
:1062B000C901DF91CF911F910F910895861797071C
:1062C00048F18C0120E030E0EF01CA1BDB0B8C179A
:1062D0009D07C0F4A9019801261B370B41095109FC
:1062E0006091060170910701809108019091090168
:1062F0000E94D3519C013058C901DF91CF911F9169
:106300000F910895EA0FFB1FE817F90758F020E0F6
:1063100030E0CECF20E030E8C901DF91CF911F916E
:106320000F910895A90198012E1B3F0B41095109B6
:1063300060910A0170910B0180910C0190910D0107
:106340000E94D3519058D6CFCF92DF92EF92FF9216
:106350001F93CF93DF931F92CDB7DEB78091E60BEB
:10636000833009F496C080916E0C833009F493C099
:1063700080916913882309F4D0C0813009F4FEC0EC
:1063800080916A1387FDF5C060E2805D0E94351A36
:1063900040E06091A21484E00E94D81980916913B2
:1063A000811164C061E08091A214882309F45EC069
:1063B00040E086E00E94D8198091E60B41E08230EF
:1063C00009F4A7C061E0811101C060E080E00E9493
:1063D000D81980916E0C41E0823009F498C061E0D8
:1063E000811101C060E081E00E94D81961E08091D4
:1063F0007F0D813009F060E040E082E00E94D81912
:1064000080917F0D41E0823009F040E061E0823010
:1064100008F460E083E00E94D81960917D13462F54
:1064200088E00E94D819409179138091781361E037
:10643000811103C0411101C060E087E00E94D819BA
:1064400080917F0D811114C08091E60B833081F023
:1064500080916E0C833061F08091691361E082302D
:1064600019F0843009F060E0462F08C060E0A0CF4A
:1064700080917E0D8823F1F161E040E085E00F908E
:10648000DF91CF911F91FF90EF90DF90CF900C9410
:10649000D81980916E0C21E030E0833011F020E0BB
:1064A00030E048E8429FC001439F900D11248A517B
:1064B000944FFC01EA57FF4F1081FC01EF57FF4F4B
:1064C00020818091F70C90E0820F911D41E080388F
:1064D00091050CF440E0612F70E080E090E049838A
:1064E0000E94071A49811436B0F4642F89E00E9493
:1064F000D8194ECF8091E60B61E0833009F4BDCF0F
:1065000080916E0C833009F4B8CF60E0B6CF40E0E4
:1065100066CF40E057CF61E0E9CF40E060E089E03E
:106520000E94D81980916D1390916E13A0916F13F2
:10653000B0917013B7FD1DC010916C131031F1F1C3
:10654000209171133091721340E050E0A4E6B0E066
:106550000E9483566C01FF24D7FCF094EF2C812F0E
:106560000E949D17811116C0C701B6010E94071A2B
:106570000FCF60E280E20E94351A0ACF6091A0142A
:106580007091A11480E090E00E94071A40E06091B1
:106590006B13ACCF82E3C81AD108D7FC19C0EE2424
:1065A000D7FCE094FE2C609172136095661F6627FD
:1065B000661F40E089E00E94D819D6CF5DDE9C01BD
:1065C000442737FD4095542F30584F4F5F4FBECF73
:1065D000D194C194D108E3CFFC0126893789468D37
:1065E000578DAA27429FB12D539FC001349FB00DF4
:1065F000811D9A1F529FB00D811D9A1F112480A3E7
:1066000091A340955095AA27429FB12D539FC00159
:10661000349FB00D811D9A1F529FB00D811D9A1F8E
:10662000112482A393A3408551856285738540839D
:106630005183628373830895FF920F931F93CF93C7
:10664000DF93EC01F62E1C821D821E821F820E89B2
:106650001F896CA17DA1CB01A0E0B0E07727662760
:10666000980140E050E00E94CE563F8F2E8FF110EF
:1066700019C084E089A719A218A2B801C9010E9413
:1066800085149BA38AA388899989AA89BB89888351
:106690009983AA83BB83FFA2DF91CF911F910F91B2
:1066A000FF90089581E089A7CE0196DFFFA2DF91D8
:1066B000CF911F910F91FF900895CF93DF93EC013D
:1066C0001C821D821E821F82188219821A821B82DE
:1066D00089A58F5F89A7833061F1853021F18230F0
:1066E00019F0DF91CF9108956E897F897DA36CA306
:1066F0008C899D890E94851499A388A36E897F89BE
:106700008C899D89809590950E9485149BA38AA36E
:106710004C855D856E857F85488359836A837B833D
:10672000DF91CF91089519A61DA21CA2DF91CF91F0
:10673000089519A218A28E899F899BA38AA3DF912D
:10674000CF910895CF92DF92EF92FF92CF93DF9394
:10675000EC01CC80DD80EE80FF808F2D9927AA2769
:10676000BB27892B8A2B8B2B09F042C089A582304D
:1067700009F433C070F5813009F444C040E050E0C2
:106780002AA13BA1AA27429FB12D539FC001349F4C
:10679000B00D811D9A1F529FB00D811D9A1F1124AB
:1067A00028A139A1820F931F9DA38CA348815981F1
:1067B0006A817B814C0D5D1D6E1D7F1D4C835D8349
:1067C0006E837F83DF91CF91FF90EF90DF90CF902A
:1067D00008958330A1F0843089F68EA1811122C002
:1067E000BB27AF2D9E2D8D2DAC0140955095C8CF68
:1067F000CE0163DFCC80DD80EE80FF80B7CF4C8997
:106800005D89BECF8EA1811105C077276F2D5E2DCA
:106810004D2DB6CF40E253E0C701B6010E94961459
:10682000AC01AECF40E251E0C701B6010E94961420
:10683000DBCFCF93DF93ECE9FBE0AEE9BBE080E098
:1068400090E05AE26FEF11C0589F9001599F300DB0
:106850001124E901C65CDE4E49A5411127C001960D
:106860003C961C9686309105F1F02081222361F33D
:10687000589FE001599FD00D1124C65CDE4E29A51A
:106880002111EDCF10821C92EF0121976883EF0157
:106890002297688320812223B9F201963C961C96A8
:1068A0008630910511F7DF91CF9108951FA21DA2A7
:1068B0001CA21C821D821E821F821F8E1E8E19A684
:1068C00019A218A21BA21AA2188219821A821B826C
:1068D000E901C25CDF4E1FA21DA21CA21C821D8208
:1068E0001E821F821F8E1E8E19A619A218A21BA21D
:1068F0001AA2188219821A821B82B1CF8091391094
:106900008E7F9091F51291118160809339100E94D1
:106910000C1180913910877F9091F8129111886045
:10692000809339100E940C11809139108D7F9091C5
:10693000F61291118260809339100E940C1180919F
:1069400039108F7E9091F9129111806180933910E6
:106950000E940C11809139108B7F9091FB12911144
:106960008460809339100E940C11809139108F7DC2
:106970009091FC1291118062809339100E940C1149
:10698000809139108F7B9091FD12911180648093DA
:1069900039100C940C11CF93DF93EC01898D90E0AA
:1069A0009927FC01E45BFE4F3491FC01E45BFD4F51
:1069B0002491FC01E45BFC4F849190E0A0E0B0E006
:1069C000DC0199278827922B28A5832B022E04C04F
:1069D000B695A795979587950A94D2F7880F991F32
:1069E000AA1FBB1F880F991FAA1FBB1F880F991FC3
:1069F000AA1FBB1F880F991FAA1FBB1F88879987D3
:106A0000AA87BB874B8D50E05527FA01E45BFE4F08
:106A10008491FA01E45BFD4F9491FA01E45BFC4F31
:106A2000449150E060E070E0BA0155274427592BAB
:106A3000482B022E04C076956795579547950A9482
:106A4000D2F7440F551F661F771F440F551F661F4F
:106A5000771F440F551F661F771F440F551F661F72
:106A6000771F4C875D876E877F874D8D50E0552758
:106A7000FA01E45BFE4F8491FA01E45BFD4F9491CF
:106A8000FA01E45BFC4F449150E060E070E0BA0131
:106A900055274427592B482B04C076956795579561
:106AA00047952A95D2F7440F551F661F771F440F4D
:106AB000551F661F771F440F551F661F771F440F12
:106AC000551F661F771F488B598B6A8B7B8B89A557
:106AD0008230A9F170F4813009F44EC019A218A2D5
:106AE0001BA21AA2188219821A821B82DF91CF91EF
:106AF00008958330B9F0843089F719A218A26E89FD
:106B00007F898E8D9F8D0E9485149BA38AA388897F
:106B10009989AA89BB8988839983AA83BB83DF91DA
:106B2000CF91089519A218A28E899F899BA38AA349
:106B3000188219821A821B82DF91CF9108956E8983
:106B40007F898C899D890E94851499A388A36E8969
:106B50007F898C899D89809590950E9485149BA33F
:106B60008AA38C859D85AE85BF8588839983AA83FA
:106B7000BB83DF91CF910895CE01DF91CF912CCDD2
:106B8000CF92EF92FF920F931F93FC01AC2DA07850
:106B9000C0FE08C0808D918D8617970719F0718F00
:106BA000608FA1E0C1FE08C0828D938D8417950788
:106BB00019F0538F428FA1E0C2FE08C084899589E5
:106BC0008217930719F0358B248BA1E0C3FE08C010
:106BD000848D958D8017910719F0158F048FA1E092
:106BE000C4FE0EC0868997898E159F0549F0F78AE5
:106BF000E68ACF011F910F91FF90EF90CF90CBCEFF
:106C0000A111F7CF1F910F91FF90EF90CF900895B2
:106C1000AF92BF92CF92EF92FF920F931F93CF93B9
:106C2000DF93F62E142F590180E00E94ED13612F9F
:106C300081E00E94E025002309F45BC080917F0D74
:106C4000811157C0FF2009F44AC020913F133091B1
:106C50004013A501AA27429FB12D539F7001349F75
:106C6000B00DE11CFA1E529FB00DE11CFA1E11245A
:106C700020953095E20EF31E5AE21502E001112430
:106C800020E1C22E00E010E020E030E040E050E0E3
:106C900060E070E0CE01825C9F4E72DF20913D1378
:106CA00030913E13A501AA27429FB12D539F700139
:106CB000349FB00DE11CFA1E529FB00DE11CFA1E6C
:106CC000112420953095E20EF31E20E030E040E0E4
:106CD00050E060E070E0CE01865C9E4E51DFDF91B7
:106CE000CF911F910F91FF90EF90CF90BF90AF90F9
:106CF00008954AE21402E00111246F2DCE01825C56
:106D00009F4E9ADC6F2DCE01865C9E4E95DC9ACF0D
:106D1000AF92BF92CF92DF92EF92FF920F93CF93F9
:106D2000DF931092E50B33E2A32E37E0B32E4DE94B
:106D3000E42E4BE0F42E5EE9C52E5BE0D52EE50196
:106D40004C2F4A1989919091E30B892341F0F70167
:106D50008081882321F0F60180818823A1F0FCE066
:106D6000EF0EF11C8CE0C80ED11CE7E0C932DE0743
:106D700039F7DF91CF910F91FF90EF90DF90CF9097
:106D8000BF90AF900895F701359720813181F701C9
:106D9000329700E060E080813BDFF7011082DFCFB7
:106DA0002F923F924F925F926F927F928F929F921B
:106DB000AF92BF92CF92DF92EF92FF920F931F9309
:106DC000CF93DF93CDB7DEB72C970FB6F894DEBF25
:106DD0000FBECDBF782E642E552E298386958695BD
:106DE000869590E0E72DE770F0E0ED5DF84F2081AB
:106DF000FC01EC57F54F662309F4C6C08081822B55
:106E00008083E72DF0E0EE0FFF1FEC56F54F408337
:106E10005183412CC090870DD090880DE090890D52
:106E2000F0908A0D8091E40B882309F409C16091E8
:106E3000E20B662359F1272D30E080E090E028171F
:106E4000390701F1E82FE695E695E695F0E0EC5775
:106E5000F54F40814423B1F0FC01E770FF27ED5D61
:106E6000F84F5081542371F0821793071CF461305E
:106E700009F471C0281739071CF4623009F46BC09B
:106E800044244394019680389105C9F640E08CED86
:106E9000A82E8BE0B82E11E0872C912CD5018D9176
:106EA0005D018F3F09F457C0242E332427FC309412
:106EB0009101220F331F220D331D220F331F220F8A
:106EC000331F2C57354FF901E85EFE4F1083F9014F
:106ED000E75EFE4F1083F901E65EFE4F1083F90175
:106EE000EC5EFE4F60825182F901EA5EFE4F7082D5
:106EF000F401E80FF11DCF01F901E95EFE4F808337
:106F0000F901E05FFE4FC082D182E282F382F90193
:106F1000E55EFE4F29812083042D262D352D61E06D
:106F200077DE2091E30B04C0242E332427FC309419
:106F3000C101019666E070E00E94E251482FFC0119
:106F4000ED5DF84F8081822379F352EEA5165BE068
:106F5000B50609F0A3CF2C960FB6F894DEBF0FBE8E
:106F6000CDBFDF91CF911F910F91FF90EF90DF90F8
:106F7000CF90BF90AF909F908F907F906F905F90D9
:106F80004F903F902F900895209580812823208353
:106F90000091E20B80E090E06FE770E0023009F4CE
:106FA0004BC09C01122FE22FE695E695E695F0E0A6
:106FB000EC57F54F4081442321F1F901E770FF2799
:106FC000ED5DF84F50815423E1F0ECE9FBE04081A6
:106FD000442339F0DF0112974C9150E042175307D8
:106FE00081F03C96ABE0E43EFA0789F7F901EE0F39
:106FF000FF1FEC56F54F60805180712E442443945E
:1070000009CF01968038910549F67EE9E72E7BE0AD
:10701000F72E10E0F70132978081882331F0F701D5
:1070200034978081871509F4A5C01F5FFCE0EF0E3F
:10703000F11C163079F78FCF9B01281B390BB2CF8B
:107040002091E30B03E217E044E95BE05B834A83B2
:107050009CE9292E9BE0392EF8014FEF88248A9471
:10706000982C5401302F1DC06D917D918D919C9174
:107070006C157D058E059F0538F4C1010197DC0173
:107080008C91781609F4D6C06A817B81645F7F4F4A
:107090007B836A837CE0270E311C87E0E932F807A6
:1070A000C1F05E2F531B8191822371F3D1018C912A
:1070B000AA81BB818111D8CF6D917D918D919C91D9
:1070C000681579058A059B05F8F64B015C01452F8B
:1070D000DBCF842F4F3F09F0DACE6AE9262E6BE032
:1070E000362EE3E2F7E088248A94982C54019E2FF0
:1070F000931B4191422301F1D1015C91A52FA695EB
:10710000A695A695B0E0AC57B54F4C91411121C062
:10711000A10146505109DA014D915D916D917C912B
:107120004A835B836C837D83481559056A057B051B
:1071300018F44A015B01892FBCE02B0E311C47E09B
:10714000E932F407A1F68F3F39F187FD04CF482FCC
:107150009ECE5770A52FB0E0AD5DB84F5C91542323
:10716000B9F2BCE02B0E311C47E0E932F40709F01C
:10717000BECFE9CFF70110828091E50B811155CF89
:1071800031971082F701339700E0262D352D412FDE
:1071900060E080813DDD49CF5091E20B5A87EBE9F9
:1071A000FBE07B8688248A94982C54018E829F82EF
:1071B000A886B98625C01F0147E0241A3108D101ED
:1071C0008D909D90AD90BC908A829B82AC82BD8256
:1071D0004E815F816885798584169506A606B70677
:1071E00048F48A819B81AC81BD818E839F83A8876F
:1071F000B9878C853C9697E00932190709F4A5CF29
:10720000902E931A9C86D8019D918D01922391F323
:10721000BA85B13051F078F2B23061F790816B8568
:10722000961740F78C859B87E5CF90815B85591732
:10723000C8F3E0CF452F2BCECF9380917B0D8F3FAE
:10724000A9F0C82FCF7780917D0D8C0F20E040E012
:1072500050E060E0885EA4DD60917D0D6C0F685E9B
:1072600040E08091A414CF910C948E12CF91089598
:107270009F92AF92BF92CF92DF92EF92FF920F93C5
:107280001F93CF93DF93182F962E80917F0D811738
:1072900009F443C0D1DF8FEF9FEF90937A0D809375
:1072A000790D8FEF80937B0D40E850E06FEF70E039
:1072B00089EF9CE00E94E45533E2A32E37E0B32E21
:1072C0004DE9E42E4BE0F42E5FE9C52E5BE0D52EB0
:1072D000E5014C2F4A1989919091E30B892341F0E4
:1072E000D7018C91882321F0F601808181115BC048
:1072F000BCE0EB0EF11CECE0CE0ED11CF7E0C93285
:10730000DF0739F780E1E4E8FAE0DF011D928A95B2
:10731000E9F71092E50B111116C0911004C080918D
:107320007E0D811129C010937F0D90927E0DDF910B
:10733000CF911F910F91FF90EF90DF90CF90BF9072
:10734000AF909F9008952091A6148FEF9FEF909398
:107350007A0D8093790D2111E0CF8091E60B823078
:10736000E1F280916E0C8230C1F28FEF9FE7909333
:107370003B1080933A10D1CFA9EFBCE0FD019FEF05
:1073800005C031968DE0E937F80749F0808187FF25
:10739000F8CF9083F6CFEDE0A937BE0799F08D9135
:1073A0008F3FC9F3C0CF379720813181F6013497E1
:1073B00000E060E080812CDCD7011C92F60131975F
:1073C000108296CF39DFAFCF0F93CF934FB7F8949A
:1073D00036EC31BB469A80EE87B997E09AB98DB901
:1073E00081E085B980E488B91BB880E28EB987E472
:1073F00081BB52E05A95F1F700C026B199B18CB12A
:1074000031BB479AC22FC695C37050E8259F9001A3
:107410001124C22B292F2071C22B292F26952695A6
:107420002870C22B96959076C92B90E0880F991FF3
:1074300084709927C82B87EE87B987EF8AB982EEC7
:107440008DB94FBF80910613882381F08091771802
:10745000C5FF2FC08C2785FD0EC08091A6148230F9
:10746000C1F0C0937718CF910F910895809177184C
:107470008C2785FFF2CF80917F0D882339F161E061
:10748000C5FD60E0F5DE0E94A4318091A614823033
:1074900041F7C0FFE6CF8091771880FDE2CF809161
:1074A000F3128E5F8093F312C0937718CF910F91F0
:1074B000089585FFCFCFC8D786E0ECEDFBE0ABE4C5
:1074C000B3E101900D928A95E1F7C7CFC5FF11C0D6
:1074D0001FDC00E04091A4144F70406BE0917B19D9
:1074E000F0917C1920E463E070E08BE799E1099565
:1074F000B4CF81E08093E50B0FE7ECCFCF93809181
:107500007F0D882399F0E9EFFCE004C08DE0E937B6
:10751000F80761F081918F3FC9F38EDE80917F0D76
:107520008230E1F0833019F1813009F1CF91089573
:10753000615071098109910960687F6F8F6F9F6F3A
:107540006F5F7F4F8F4F9F4FFB0170937A0D60935A
:10755000790DE750F34F80818F3F21F50E94485607
:107560006F7777278827907897FFEECFE1CF20912C
:10757000790D30917A0D07C09C01FC01E750F34F63
:1075800040814F3F59F4C90101968F77907897FF5A
:10759000F3CF019780689F6F0196EECF8093790DAE
:1075A00090937A0DC081CF7780917C0D885E20E02A
:1075B00040E050E861E08C0FF3DB80917C0D885E49
:1075C00060E070E88C0F0E947512E091790DF091E7
:1075D0007A0DE750F34F808180937B0D80917C0D75
:1075E00080937D0DCF910895BF92CF92DF92EF925D
:1075F000FF920F931F93CF93DF938C017C0181E85F
:10760000E80EF11CF70180818823B9F1E801CC571D
:10761000DF4F8881998197FD30C0F801E80FF91F8D
:1076200081816801F7E8CF0ED11C22C078E1B72E26
:10763000B80EF6018081B80E20E040E050E060E036
:107640008B2DAEDB40E06B2D8091A4140E948E1236
:10765000888199810196F701608170E00E94E25172
:1076600099838883F801E80FF91F818187FF05C09E
:107670008F73982F9E539230C8F6DF91CF911F9150
:107680000F91FF90EF90DF90CF90BF9008958F9271
:107690009F92AF92BF92CF92DF92EF92FF920F93A1
:1076A0001F93CF93DF931F92CDB7DEB700E010E0BA
:1076B000F8E8BF2EB09E4001B19E900C112486EEDA
:1076C0009BE0880E991ED4018C91823099F00F5F57
:1076D0001F4F0230110571F70F90DF91CF911F916D
:1076E0000F91FF90EF90DF90CF90BF90AF909F9061
:1076F0008F9008956401B1E8CB0ED11CF601808112
:10770000882329F37401F2E8EF0EF11CD701ED9103
:10771000FC91E80DF91D41814E33B1F0C40149835C
:1077200063DF4981842F8E53823070F0F401EC576F
:10773000FF4FD7012D913C91318320838091F60C2E
:10774000F401E957FF4F80834F73842F8E538230AB
:1077500088F0E8E1AE2EA40E8091F60CA80E20E091
:1077600040E050E861E08A2D1BDB60E070E88A2D84
:107770000E947512F701808191810196D6016C916A
:1077800070E00E94E25191838083F401E80FF91FB9
:10779000418147FDD9CF9BCF842F2091A31427FD92
:1077A00009C06F7070E0332727FD309562177307AB
:1077B00009F0089520E040E050E060E0F1CA842F35
:1077C000E091A314E7FD09C06F7070E0FF27E7FDAB
:1077D000F0956E177F0709F00895422F50E0542F5F
:1077E0004427550F41505E4F61E0211101C060E018
:1077F00020E0D6CA6F928F929F92AF92BF92CF92A3
:10780000DF92EF92FF920F931F93CF93DF93E0915C
:107810009B19F0919C19309719F08BE799E1099524
:1078200083E69AE10E94BE24082F10E0011511059D
:1078300009F478C0C0E0D0E09091631A2091651AF5
:10784000EE24E394F12CE3E09E2EF4E08F2EA2E0F0
:10785000AA2EBB24B394892F622F90E070E00E947F
:10786000E251E091661AF091671AE80FF91FF08172
:10787000F83F08F065C0F7FF71C08091A01984300F
:1078800031F0F0939D19F092A219E092A1198F2F77
:10789000807F803B79F198F4803961F1803A51F131
:1078A000803841F1F03F09F4B1C0F73F09F4C3C09B
:1078B0001092A0191092A2191092A1191DC0803D1A
:1078C00009F4A1C008F49CC0803EA1F0803F51F7AC
:1078D000EF2FE15FEF3030F7AE2FB0E0A15BB84F94
:1078E0008C91813009F49BC0E8F2823009F48BC09E
:1078F0008330F1F69092A0193FB7F8949091631AF3
:10790000892F90E001962091651A622F70E00E9405
:10791000E251982F8093631A3FBF2196C017D10779
:1079200008F499CFDF91CF911F910F91FF90EF90C5
:10793000DF90CF90BF90AF909F908F906F90089501
:10794000D090A019B092A01920E040E06F2F81E004
:1079500090E00E94A112D092A019CECF6090A01901
:10796000662051F24091A1195091A2199A01ABEAF7
:10797000BAEA0E94C2566C01D694C794C601880F19
:10798000991F8C0D9D1D6A01C81AD90AD601A558E8
:10799000B64E9296FC93CA0101969093A2198093D9
:1079A000A11921E0C216D104B9F022E0C216D10417
:1079B00009F0A2CF20919F1940919E1960919D19C5
:1079C0000E94A1128091A019843009F495CFF09201
:1079D000A219E092A11990CF22E062128DCF20E08F
:1079E00040919E1960919D190E94A1128091A01949
:1079F000843009F481CFD092A219C092A1197CCF12
:107A0000803C09F04FCFA092A01976CF8092A019A8
:107A1000F0939D19F092A219E092A1196DCF809375
:107A2000A01920E040E06F2F81E090E00E94A112B9
:107A30001092A01961CF4091A1195091A2199A01F9
:107A4000ABEABAEA0E94C256969587959C01220F2E
:107A5000331F280F391FDA01A21BB30BA558B64EEE
:107A60009296FC93CA0101969093A2198093A11952
:107A700020919F1940919E1960919D190E94A11219
:107A80001092A01939CFCF93C82F6C2F80E89DE0BA
:107A90000E94932481110FC080E89DE00E94BE24C3
:107AA000882399F30E9453126C2F80E89DE00E9476
:107AB0009324882389F3CF910895EF92FF920F9337
:107AC000CF93DF931F92CDB7DEB77B0161157105B0
:107AD00039F40F90DF91CF910F91FF90EF900895BF
:107AE000842F2983D0DF298182E0E816F10488F30E
:107AF000822FC9DFE2E0EE16F10459F3802F0F90D8
:107B0000DF91CF910F91FF90EF90BDCF6F927F9259
:107B10009F92AF92BF92CF92DF92EF92FF920F931C
:107B20001F93CF93DF931F92CDB7DEB719EF612E6E
:107B30001FE0712E60E008E010E086ECC82EDD2426
:107B4000D39490EFB92E27E8E22EF3018191919121
:107B50003F01B8EFFB2EF62A262F2695269526956F
:107B6000A80102C0440F551F2A95E2F7942E909465
:107B70009F20AFB6F89469830E94940EC1BA469ACA
:107B80003F2D330F367031649F2D96959270906A19
:107B9000D5B838B9BBB89EB9E1BA55E05A95F1F7F6
:107BA0000000C1BA469A792D770F492D4695592D77
:107BB000551F5527551F872F8670582B5064292D28
:107BC0002071872F880F8072822B707C872B4270E8
:107BD000406AD5B858B98BB94EB9E1BA8AE08A95EE
:107BE000F1F700C0C1BA469AD5B838B9BBB89EB94A
:107BF000E1BAEAE0EA95F1F700C0AFBE69816F5FD4
:107C0000603209F0A2CF0F90DF91CF911F910F91B9
:107C1000FF90EF90DF90CF90BF90AF909F907F90BC
:107C20006F900C940C11CF93DF931092470A10922F
:107C3000480A1092440A1092430A1092460A10927F
:107C4000450A10924D0A40E061E088E00E94D81990
:107C50001092301010922F1059DF2FEF82E597E02D
:107C6000215080409040E1F700C00000C9E3D0E11E
:107C700088818E7F88830E940C1188818D7F888304
:107C80000E940C118881877F88830E940C11888153
:107C90008F7E88830E940C1188818F7D88830E944B
:107CA0000C1188818F7B88830E940C1188818B7FC7
:107CB00088830E940C111092361010923510109289
:107CC000321010923110109238101092371010921A
:107CD0002A1010922910109234101092331060E381
:107CE00083E00E94321160E783E00E94321162EB70
:107CF00083E0DF91CF910C94321160918B0D66304F
:107D000090F06C3040F06B5D86E60E94351A81E0A1
:107D10000E94FF0FFBCE655D82E60E94351A81E06E
:107D20000E94FF0FF3CE6F5C81E60E94351A81E05E
:107D30000E94FF0FEBCECF92DF92EF92FF92CF9394
:107D4000DF93D82FC9E1D9DFC150E9F71092791834
:107D5000109278186AE081E10E9478110E945C110B
:107D6000C12CD12C760134C060E082E00E947811F1
:107D700061E088E00E94781180E00E94A81160E133
:107D800081E00E94781181E00E94A81160E080E10A
:107D90000E94781180E00E94FF1160E180E00E9463
:107DA000781160E080E10E94781181E00E94FF116B
:107DB0006AE080E00E947811D1500E945C11C80EE8
:107DC000D91EE11CF11C99DF80917A18853058F496
:107DD000D111CACFB601C701DF91CF91FF90EF90CB
:107DE000DF90CF900895CC24CA94DC2C7601F2CF9A
:107DF0002F923F924F925F926F927F928F929F92BB
:107E0000AF92BF92CF92DF92EF92FF920F931F93A8
:107E1000CF93DF93CDB7DEB72D970FB6F894DEBFC3
:107E20000FBECDBF682E6C83542E10927A1870E06E
:107E300080E090E00E9426539B01AC0160E070E07E
:107E400080E090E40E940D5524EA30ED42E851E4D0
:107E50000E94AA549B01AC0160E074E284EF99E4B3
:107E60000E9461521B01482E9983862D90E09F83CA
:107E70008E832C81235081E090E0022E01C0880F78
:107E80000A94EAF78D837EE0772E00E010E8EE2476
:107E9000EA94FE2CAE81BF81AA0FBB1FA750B04F42
:107EA000BB83AA83E22FFF27E1950CF4F0954F01E5
:107EB000AA2497FCA094BA2CFD86EC860AC0EC8517
:107EC000FD85E00FF11FFD87EC87169507957A94E5
:107ED00031F1462D60E0852D0E9403182C853D85EB
:107EE0008217930708F44EC06FEF7FEF8FE79FE78D
:107EF000262F372F482F592FF980622D732D842D6F
:107F00009F2D0E945A5287FDDACF2C853D85201B7C
:107F1000310B3D872C87169507957A94D1F6EC8422
:107F2000FD848C8190E0880F991FFC01EE0FFF1FEC
:107F3000EE0FFF1FEE0FFF1FE80FF91F8E819F81CD
:107F4000E80FF91FEE0FFF1FE258FC4EF182E082AE
:107F500080E02D960FB6F894DEBF0FBECDBFDF9147
:107F6000CF911F910F91FF90EF90DF90CF90BF9036
:107F7000AF909F908F907F906F905F904F903F90C9
:107F80002F900895AA81BB812D933C938D81D3DEE0
:107F90006B017C016F3FBFEF7B078B079B0729F1CC
:107FA000C501B4010E9428539B01AC0160E070E060
:107FB00080E090E40E940D55562F472F382F292F2F
:107FC000C701B6012B873A87498758870E942653F5
:107FD000588549853A85F32E2B85E22F252F342F9E
:107FE0004F2D5E2F0E94AA5483CF8FEFB2CF0F93F5
:107FF0001F93CF93DF93182F80938B0DC62FD0E064
:108000002296DE01AA0FBB1FAB50B04F2FEF3FEF00
:108010002D933C938C3008F062C003E04CE0602F5D
:10802000812FE6DE811103C00F5F0730B9F7E12F22
:10803000F0E0DF01AA0FBB1FA651BC4E4D915C9131
:10804000CA01880F991FDF01AA0FBB1FA25FBB4E99
:108050002D913C91821B930BDF01AA0FBB1FAA53EA
:10806000BC4E8D939C939C01220F331F241B350B18
:10807000DF01AA0FBB1FAE55BC4E2D933C93220FC0
:10808000331FDF01AA0FBB1FA258BC4E281B390BA0
:108090002D933C93AF01440F551F46585B4ECF01C3
:1080A000880F991F8A5A9B4EDC018D919C91880FF5
:1080B000991FEE0FFF1FEE5CFB4E20813181821B6A
:1080C000930BFA0191838083CC0FDD1FCB50D04FEF
:1080D00019821882DF91CF911F910F9117CD04E083
:1080E00044E2602F812F84DE811103C00F5F0830CE
:1080F000B9F7E12FF0E0EE0FFF1FE25FFB4E43E028
:10810000DF01949720813181220F331F84A195A133
:10811000281B390B11963C932E934150FD014F3F84
:1081200079F7D2CF3F924F925F926F927F928F9268
:108130009F92AF92BF92CF92DF92EF92FF920F93F6
:108140001F93CF93DF93CDB7DEB768970FB6F89440
:10815000DEBF0FBECDBF082F30906C13C0908F0FC5
:10816000D090900FE090910FF090920F80910E01BF
:1081700090910F0120911201309113014090100154
:10818000509011015201A094B094AC01421B530BCA
:108190005E834D83A20160E070E04F83588769875A
:1081A0007A874091140150911501609116017091E8
:1081B00017014B875C876D877E874901880E991E62
:1081C000B40180E090E06F87788B898B9A8B8091E7
:1081D000180190911901A0911A01B0911B018B8B8C
:1081E0009C8BAD8BBE8B90916B1310E0632C77242E
:1081F00067FC7094C982DA82EB82FC8275011EC032
:10820000F301EE0FFF1FED54F04FC080D1800E94AC
:108210009D17882339F0EC14FD0408F051C0CC24DC
:10822000CA94DC2CEF89F88DEE0FFF1FE15FFC4E46
:10823000D182C08291E01F5F1E3119F1A12EB12CB5
:10824000B88EAF8AF501EF5CF84F80818F3F99F3CC
:10825000011131C08315A1F2E82FFF27E7FDF0954A
:1082600049815A816B817C81082E04C0769567957F
:10827000579547950A94D2F740FDC3CF1F5F1E3133
:10828000E9F690936B1368960FB6F894DEBF0FBEB5
:10829000CDBFDF91CF911F910F91FF90EF90DF90B5
:1082A000CF90BF90AF909F908F907F906F905F9096
:1082B0004F903F900895E82FFF27E7FDF095A1CF5D
:1082C000C414D504D0F0C601A0E0B0E0AD80BE80FB
:1082D000CA14DB04A8F49C01AD01AF80B884C98442
:1082E000DA842A193B094C095D096B857C858D85EB
:1082F0009E850E94D3516C0195CFC12CD12C92CF79
:108300008C149D0420F0C12C90E8D92E8BCF9C01B9
:10831000AD01AF84B888C988DA882A193B094C09AD
:108320005D096B897C898D899E890E94D351905803
:108330006C0178CFBF92CF92DF92EF92FF920F93B2
:108340001F93CF93DF938C01BFB6F89401501109AE
:1083500015950795159507950F5F1F4F80EF93DBD8
:1083600080E091DB81E68FDB86E18DDB81E08BDBDA
:10837000101611068CF5C0E0D0E0FE01EE0FFF1FD5
:10838000EE0FFF1FEF51F94EC080E180D280F380E5
:108390008C2D8F7778DB8E2D8F7775DB8D2D8F77FA
:1083A00072DB8F2D8F776FDB9D2D92959695947054
:1083B0003E2D3295369536953270932B2F2D229582
:1083C0002870922B8C2D881F8827881F892B5BDBB8
:1083D0002196C017D1078CF287EF55DBBFBEDF9126
:1083E000CF911F910F91FF90EF90DF90CF90BF90B2
:1083F0000895882349F080E89DE00E94BE24811101
:1084000001C008950C945312F5D9F5CFCF93DF93A3
:1084100000D000D000D0CDB7DEB786E0EBE2F7E0C9
:10842000DE01119601900D928A95E1F760E0CE0190
:1084300001960E94512426960FB6F894DEBF0FBE17
:10844000CDBFDF91CF910895CF93DF9300D000D0BF
:1084500000D0CDB7DEB746E050E06FEF70E0CE0160
:1084600001960E94E45540E080E090E00AC0298136
:10847000321B30834F5F46303CF5019680389105C2
:1084800019F1382FE82FE695E695E695F0E0EC57E0
:10849000F54F2081222389F3FC01E770FF27ED5D72
:1084A000F84F5081522349F3E1E0F0E0EC0FFD1F5B
:1084B000E40FF11D47FDFA9580834111D8CF41E0CB
:1084C000019680389105E9F661E0CE0101960E949F
:1084D000512426960FB6F894DEBF0FBECDBFDF91B4
:1084E000CF9108956F927F928F929F92AF92BF9299
:1084F000CF92DF92EF92FF920F931F93CF93DF9370
:108500001F92CDB7DEB7C62EE82EFF24E7FCF0940D
:10851000282F38E82303800111240A51144FD80171
:108520008C916817E9F09091E60BDD24D39492309A
:1085300029F090916E0C923009F0D12C882301F132
:10854000833009F409C1823009F43BC1B2E0CB1693
:1085500009F455C0E3E0CE1609F4E4C0D801CC928A
:108560000F90DF91CF911F910F91FF90EF90DF90CF
:10857000CF90BF90AF909F908F907F906F90089515
:108580005801BFEFAB1ABB0A9FB6F89461E0C70170
:1085900088539F4F0E941516882309F404C138019F
:1085A000E1E86E0E711CE0918C0FF0918D0F8191BE
:1085B000F0938D0FE0938C0FD5018D935D01A6157F
:1085C000B705A9F79FBEF3011082D801AA57BF4F84
:1085D0001C9280E006C08F5FF3018083803809F42D
:1085E000B5CFF801E80FF11D918197FD03C02C91E3
:1085F0002F5F2C939F3F79F7B2E0CB12ABCFC090A7
:10860000A61488E88E9DF0018F9DF00D1124EA518B
:10861000F44F8081823009F4D8C028E82E9DC00133
:108620002F9D900D11248A51944FFC01EE57FF4F5E
:1086300011821082FC01EC57FF4F2FEF3FEF318387
:108640002083CC2009F473C082E0F80180838091FC
:108650003C1090913D10DD2009F482CF8F3FBFEF99
:108660009B0709F47DCF9695879520913A1030911C
:108670003B102817390708F073CF3801E1E86E0E78
:10868000711CD3018C91882309F46ACF7801B2E878
:10869000EB0EF11CD701ED91FC91E00FF11F218150
:1086A0002E33B9F0C80129830E94F43A2981822F20
:1086B0008E53823070F0F801EC57FF4FD7018D9147
:1086C0009C91918380838091F60CF801E957FF4FCC
:1086D00080832F73822F8E53823090F088E1D82EC2
:1086E000D20E8091F60CD80E20E040E050E861E018
:1086F0008D2D0E94D03660E070E88D2D0E9475129D
:10870000F701808191810196D3016C9170E00E9404
:10871000E25191838083F801E80FF91F218127FD41
:10872000D8CF1ECF1092F70CD801CC9219CF8091E0
:10873000E60B823009F488CF80916E0C823009F408
:1087400083CF80917F0D81117FCF8FEF9FE7909333
:108750003B1080933A1078CF4801FFEF8F1A9F0AA1
:10876000BFB6F8940E948017E0918C0FF0918D0FA6
:10877000C8018F579F4FD4012D914D012083E09167
:108780008C0FF0918D0F3196F0938D0FE0938C0F3D
:10879000A817B90781F761E0C70188539F4F0E946E
:1087A000321BBFBED3CE9FBE40E850E06FEF70E0FB
:1087B000C5010E94E45531E8632E712C600E711ED4
:1087C00002CFC8010E94F43AC1CEC8010E94F43A17
:1087D00024CFEF92FF921F93CF93DF9300D0CDB7BA
:1087E000DEB71FB7F89489839A830E948017E091BF
:1087F0008C0FF0918D0F40E09A818981A42FB0E019
:10880000AA0FBB1FA15FBC4E2D913C9121933193C8
:108810004F5F493199F7E0938C0FF0938D0F2091C2
:108820000E132093051320E0A22FB0E0AB50BD4EF5
:108830003C913083E0918C0FF0918D0F3196F09345
:108840008D0FE0938C0F2F5F273171F7A42FB0E0CD
:10885000AA0FBB1FA15FBC4E2D913C912193319378
:108860004F5F4E3199F7E0938C0FF0938D0F20916D
:108870000C132083E0918C0FF0918D0F9F012F5FDF
:108880003F4F30938D0F20938C0F20910D13218338
:10889000E0908C0FF0908D0F2FEFE21AF20AF09219
:1088A0008D0FE0928C0FEBE4F3E12191D7012C9333
:1088B000E0908C0FF0908D0FBFEFEB1AFB0AF09257
:1088C0008D0FE0928C0F23E1E135F20771F72091D3
:1088D000491330914A133093AA142093A914B70175
:1088E000E1E5F3E141915191DB014D935D93BD01D0
:1088F000B3E1E936FB07B1F7D7015896B0938D0F76
:10890000A0938C0F61E00E94321B1FBF0F900F904D
:10891000DF91CF911F91FF90EF9008952F923F929A
:108920004F925F926F927F928F929F92AF92BF927F
:10893000CF92DF92EF92FF920F931F93CF93DF932B
:10894000CDB7DEB7CD59D1090FB6F894DEBF0FBE53
:10895000CDBF803F51F1873FA9F02091850D309127
:10896000860D2639F1E03F070CF047C0A9014F5FA3
:108970005F4FF901EF51F94E80835093860D40937C
:10898000850D21C08091E116813009F4B2C08111BA
:1089900039C08091E216813609F4B3C31092860D76
:1089A0001092850D0E94C2210EC01092860D109269
:1089B000850D86E991E0E1EEF6E1DF019C011D9273
:1089C00021503040E1F7C356DF4F0FB6F894DEBFB9
:1089D0000FBECDBFDF91CF911F910F91FF90EF9010
:1089E000DF90CF90BF90AF909F908F907F906F90CF
:1089F0005F904F903F902F90089541E050E020E02D
:108A000030E0B7CF8E3751F68091E316883031F6DB
:108A10008091E416813011F68091850D9091860D3C
:108A20008639914009F0BACF08EF16E171E5E72EDB
:108A300073E1F72ED12C19C02BEA3AEA4AEA55E441
:108A4000692D7A2D8B2D9C2D0E94AA540E94FA52DA
:108A5000D7016D937C930D5F1F4FD394B2E0EB0E63
:108A6000F11CE0E8DE1609F499CFF8013197C080D7
:108A7000D8017C90F80132976081BBE0BD1558F3B6
:108A800070E080E090E00E9426534B015C01672D6E
:108A900070E0E0E8CE9E600D711D112480E090E052
:108AA0000E94265320E030E048EC5BE30E94AA5489
:108AB0009B01AC01C501B4010E94F651962EA72E70
:108AC000B82EC92E20E030E0A9010E945A5287FD3D
:108AD00015C320E030E040E451E4692D7A2D8B2D60
:108AE0009C2D0E94365418160CF0A6CF6FEF7FEF26
:108AF000AFCF8091E216823009F050CF8091850D82
:108B00009091860D839709F049CF8091E3168436C2
:108B100008F044CFE5EEF6E1DE01AB58BF4F8D0122
:108B2000208160E1269F90011124BF0161507109ED
:108B3000DB019C919F70922BD8019D938D01329601
:108B4000B7E1E530FB0761F7EB96EFADEB972E2F22
:108B50002295269526952370EC967FADEC97972F5E
:108B60009F70990F990F922B392F330F330F20E0FD
:108B70006901C094D094EA966FADEA97962E9694C8
:108B8000990C990CE996BFADE9979B2F9695969510
:108B90009695BB24B394B622B294BB0CA0EEBA2235
:108BA000B92ABB0CBB0C661F6627661F9E2F9F73DE
:108BB000990FF92EF62AE12CE0E8FE1AE6966FAD41
:108BC000E697962F990FC456DF4F9883CC59D04023
:108BD000CE57DF4F2880C258D040922D9E7FC3567B
:108BE000DF4F9883CD59D04072957F70ED969FAD41
:108BF000ED9717E0A12EA922A29400EFA022A72AA8
:108C0000E92FE695E695E695EE967FADEE97972FE0
:108C100091709295990F907E9E2B990F990FE72F47
:108C2000EE0FEE0F1E2F187700E01058F72FF29579
:108C3000F695F770EF967FADEF97E72FE170EE0FA7
:108C4000EE0FEE0FEF2BF0E0E25AF84FA081CA567C
:108C5000DF4FA883C659D040872E8694829440EF78
:108C60008422F72FF295F695F770C158DF4F78817F
:108C7000CF57D040E72FE170EE0FEE0FEE0FEF2B46
:108C8000F0E0E25AF84FA081C956DF4FA883C759D8
:108C9000D040E72FE695EF70F0E0E25AF84FA08160
:108CA000C856DF4FA883C859D04072957695777023
:108CB000C058DF4FA881C058D040EA2FE170EE0FB6
:108CC000EE0FEE0FE72BF0E0E25AF84F7081C75637
:108CD000DF4F7883C959D0407A2E7694729450EF42
:108CE00075227A2F729576957770CF57DF4FA881CE
:108CF000C158D040EA2FE170EE0FEE0FEE0FE72BD8
:108D0000F0E0E25AF84F7081C656DF4F7883CA59B7
:108D1000D040EA2FE695EF70F0E0E25AF84F70810C
:108D2000C556DF4F7883CB59D040661F6627661F34
:108D3000E796EFADE797FE2FF770FF0FF62B7F2F2B
:108D4000770F770F770F60E02B01F0E85F1A7E2F27
:108D5000771F7727771FE8966FADE897FFE36F2EB1
:108D60006622660C672A660C3E2E36947CE3372218
:108D70006295669566956370B770BB0FBB0FB62B97
:108D8000E0E1BE9FB0011124C957DF4F79836883AA
:108D9000C758D040A295A695A770E22DE170EE0FBE
:108DA000EE0FEE0FEA2B60E070E029F07E2F770FD8
:108DB000770F60E07054CC57DF4FF881C458D04033
:108DC0004F2F4170C757DF4F4883C958D040F1FB40
:108DD000552750F9C657DF4F5883CA58D040CD5752
:108DE000DF4FE881C358D0404E2F4170C557DF4F49
:108DF0004883CB58D040F3FB552750F9C457DF4F79
:108E00005883CC58D040F4FB442740F9C357DF4F78
:108E10004883CD58D040E1FB552750F9C257DF4F6A
:108E20005883CE58D040F2FB442740F9C157DF4F5A
:108E30004883CF58D040F5FB552750F9C057DF4F36
:108E40005883C059D040F6FBFF27F0F9CF56DF4FCB
:108E5000F883C159D040E4FB442740F9CE56DF4F98
:108E60004883C259D040E6FB442740F950E0440F04
:108E7000551FE7FB552750F9550F550F542BE5FBB0
:108E8000442740F9542BE3FB442740F9CD56DF4FEC
:108E90004883C359D040E2FF03C242E0242ECC579E
:108EA000DF4F4881C458D04047FB442740F9CC5697
:108EB000DF4F4883C459D0404FB7CB56DF4F48836C
:108EC000C559D040F89444E7E5EFF2E1DE01119690
:108ED00001900D924A95E1F7C757DF4F4881C95875
:108EE000D0404093F512C657DF4F4881CA58D04052
:108EF0004093F612C557DF4F4881CB58D04040937E
:108F0000F712C457DF4F4881CC58D0404093F81235
:108F1000C357DF4F4881CD58D0404093F912C25714
:108F2000DF4F4881CE58D0404093FA12C157DF4FEF
:108F30004881CF58D0404093FB12C057DF4F488143
:108F4000C059D0404093FC12CF56DF4F4881C159E1
:108F5000D0404093FD12CE56DF4F4881C259D040D9
:108F60004093FE121092FF1250930013CD56DF4F24
:108F70005881C359D040250E20920113109202133C
:108F800041E04093031310920413CC56DF4F5881F5
:108F9000C459D040509306131092071353E05093D6
:108FA00008134093091352E050930A1340930B1394
:108FB00040930E1310920F1390921013D09212132D
:108FC000C092111310921313C456DF4F4881CC592D
:108FD000D0404093141310921513B092161330938F
:108FE00018132093171310921913C356DF4F58818B
:108FF000CD59D04050931A13F0921C13E0921B13DA
:1090000010921D13A0921E1310921F139093201301
:10901000109322130093211310922313CA56DF4F8B
:109020009881C659D04090932413109225138092B2
:10903000261310922713C956DF4F2881C759D040F5
:109040002093281310922913C856DF4F3881C8592E
:10905000D04030932A1310922B13C756DF4F48810C
:10906000C959D04040932C1310922D1370922E1397
:1090700010922F13C656DF4F5881CA59D0405093D3
:10908000301310923113C556DF4F9881CB59D04021
:10909000909332135092341340923313109235133D
:1090A000609236131092371330923813C957DF4F3E
:1090B00028813981C758D04030933A13209339130F
:1090C00070933C1360933B1310923E1310923D1328
:1090D0001092401310923F1390E07BDB84E7FE0177
:1090E0003196A5EFB2E101900D928A95E1F7CB564A
:1090F000DF4F3881C559D0403FBF50CC60E070E0B1
:10910000A7CC8091E316863109F048CC8091E41613
:109110008130E1F0823009F041CC8091E516CB57E7
:10912000DF4F19821882C558D040843608F036CCFB
:10913000BE016B577F4F90E00E94A416CB57DF4FC4
:1091400088819981C558D040F5D828CC8091850D6B
:109150009091860D049765E070E00E94E251C95736
:10916000DF4F79836883C758D04077FD9BC0A5EE59
:109170008A2EA6E19A2EB6EEAB2EB6E1BB2E17EEE6
:10918000C12E16E1D12E08EEE02E06E1F02E1B01D5
:10919000220C331C220C331C260E371E49E0240EF1
:1091A000311C04E010E094E0492E512CF1EE6F2EBA
:1091B000F6E17F2E600E711E44E050E0B301C20163
:1091C0008F51994E0E94D355D30114962C91B0E83B
:1091D0002B9FC0011124F4019081982B9083922F32
:1091E00092709295990F990F907CD5018C91982B44
:1091F0009C93922F94709295990F907EF6018081A6
:10920000982B9083822F88708295807FD7019C91C4
:10921000892B8C93B4E04B0E511C0B5F1F4FE4E085
:109220008E0E911CF4E0AF0EB11C24E0C20ED11CD6
:1092300034E0E30EF11C0215130509F0B7CFC9574E
:10924000DF4F28813981C758D0402E5F3F4F220F12
:10925000331F220F331FE090E516FFB6F894ECE8B9
:10926000FDE040E052E0DF01BA011D926150704024
:10927000E1F789010550110926EE36E1A801B9018F
:10928000CF010E94CA550457124F10938D0F0093BF
:109290008C0F61E08E2D90E00E94321BFFBE7ECBD2
:1092A000212CFDCD24E030E0D6CFEF92FF920F933A
:1092B000CF93DF931F92CDB7DEB77B016091850D11
:1092C0007091860D6115710529F0E61AF70A81E0A3
:1092D000E81AF108E114F10439F40F90DF91CF910D
:1092E0000F91FF90EF900895842F298317DB298138
:1092F000E2E0EE16F10488F3822F10DBF2E0EF16C5
:10930000F10459F3802F0F90DF91CF910F91FF90CF
:10931000EF9004CB1F920F920FB60F9211240F9073
:109320000FBE0F901F9018951F920F920FB60F92BD
:1093300011240F900FBE0F901F9018951F920F923F
:109340000FB60F9211240BB60F922F933F934F93AA
:109350005F936F937F938F939F93AF93BF93CF93BD
:10936000DF93EF93FF9334997CC0CFB7F89456EC1A
:1093700051BB469A70EE77B967E06AB97DB915B806
:10938000D0E8D8B96BB91EB8B7E4B1BB82E08A9512
:10939000F1F700C026B199B18CB151BB479A422F69
:1093A00046954370E0E82E9F90011124422B292F0F
:1093B0002071422B292F269526952870422B9695B1
:1093C0009076492B90E0880F991F84709927482B3D
:1093D000A7EEA7B9F7EFFAB9E2EEEDB985E08A9505
:1093E000F1F7000047FF54C040FF52C051BB469AFE
:1093F00077B96AB97DB915B8D8B96BB980E28EB9B9
:10940000B1BB82E08A95F1F700C026B199B18CB169
:1094100051BB479A622F6695637050E8259F900173
:109420001124622B292F2071622B292F2695269536
:109430002870622B96959076692B90E0880F991F83
:1094400084709927682BA7B9FAB9EDB985E08A9598
:10945000F1F7000044FD1AC083E69AE10E949324CC
:10946000CFBFFF91EF91DF91CF91BF91AF919F91CE
:109470008F917F916F915F914F913F912F910F90BD
:109480000BBE0F900FBE0F901F9018950E94A02941
:10949000CFBFE7CF1F920F920FB60F9211240BB6DA
:1094A0000F922F933F934F935F936F937F938F937D
:1094B0009F93AF93BF93CF93DF93EF93FF93CEE64A
:1094C000D0E088818D7F888385B3876085BB789461
:1094D0000E944602F894888182608883FF91EF9110
:1094E000DF91CF91BF91AF919F918F917F916F91BC
:1094F0005F914F913F912F910F900BBE0F900FBE38
:109500000F901F901895CF93DF93CDB7DEB760977C
:109510000FB6F894DEBF0FBECDBF20E820936100E8
:1095200010926100F89414B817B81AB81DB810BAA0
:1095300015B880EE88B91BB81EB893EE91BB0FEF3B
:1095400004B987B937E03AB98DB990BB9CE797BDAC
:1095500094B5926094BD95B5936095BD90916E0061
:10956000926090936E00EC9A96EC91BB469A87B904
:109570003AB98DB915B828B91BB81EB887E481BBB4
:1095800032E03A95F1F700C086B189B18CB191BB58
:10959000479A87EE87B987EF8AB982EE8DB987EB54
:1095A00092E0EEE3F0E1DF01AC011D92415050404A
:1095B000E1F7E3ECF9E0DF011D922A95E9F781E498
:1095C000E3E4FAE0DF011D928A95E9F710E21093D7
:1095D000520A85E4E5EFFFE0DF011D928A95E9F785
:1095E00086E6EFE8FFE0DF011D928A95E9F7009338
:1095F000F40F0E94AE1782E691E0E4E8FAE0DF01A2
:109600009C011D9221503040E1F78FE38093E30BE2
:1096100046E050E06FEF70E08CED9BE00E94E45577
:109620001092DC0B0E94A02983E191E0E6EEFBE0C2
:10963000DF019C011D9221503040E1F740E850E0ED
:109640006FEF70E087EE9BE00E94E45540E850E049
:109650006FEF70E08FE69CE00E94E45587E8E9EF49
:10966000FCE0DF011D928A95E9F740E850E06FEFDA
:1096700070E0CF010E94E4558FEF9FEF90937A0D39
:109680008093790D00937B0D85E1E9E6F3E1DF013D
:109690001D928A95E9F700936A1300936C138FEF7C
:1096A0009FEFDC0180936D1390936E13A0936F1363
:1096B000B093701381E080936B1300937713009342
:1096C0007B131092A0191092A2191092A11980EC8C
:1096D0008093651A83EA99E19093671A8093661ADA
:1096E0001092641A1092631A1092841910928319BE
:1096F000109288191092871910928C1910928B1958
:1097000010928E1910928D191092901910928F1933
:109710001092941910929319109298191092971907
:1097200010929A191092991910929C1910929B19E3
:109730008DE59DE390937C1980937B198FED9BE3DE
:109740009093801980937F198CEC9BE390938219FE
:109750008093811982E093E290937E1980937D1922
:1097600087E292E290938A198093891987EF9EE1AC
:10977000909386198093851985E599E490939619BD
:109780008093951988ED93E29093921980939119A3
:109790001092860D1092850D1093820D8BEA94E144
:1097A0009093840D8093830D1092810D1092800D03
:1097B00080E090E06AE2689F9001699F300D11247B
:1097C000A901465C5E4EDA01462F1D924A95E9F7E3
:1097D000225C3F4ED901262F1D922A95E9F701966A
:1097E0008630910541F786E392E10E94881981E570
:1097F00092E10E94881981E080936B12809151124E
:1098000090915212A0915312B0915412892B8A2B2D
:109810008B2B51F46091870D7091880D8091890D8B
:1098200090918A0D0E944B560E94485660935112A7
:109830007093521280935312909354128091691234
:10984000843011F184E08093691281E592E10E94F5
:109850004414A0916A12BB27A1950CF4B095AA0FED
:10986000BB1F11962091591230915A1240915B12F0
:1098700050915C120E948D5660935D1270935E123F
:1098800080935F129093601286EC81BB469A90EEB3
:1098900097B927E02AB99DB991E095B990E498B9B4
:1098A0001BB890E29EB997E491BB32E03A95F1F78C
:1098B00000C096B199B12CB181BB479A87EE87B9A8
:1098C00087EF8AB982EE8DB994FD6DC28BED90E081
:1098D0000E94DD16811106C00E9496158BED90E066
:1098E0000E94E9431FB7F89462E08CED90E00E947B
:1098F0001516882309F455C28FE38093A51410929E
:10990000A7141092A81480E090E89093AA14809372
:10991000A91460918E0F662309F499C080918C0F71
:1099200090918D0FFC0120E030E074E2729FD00135
:10993000739FB00D1124A258BC4E6F0144E2C40EB7
:10994000D11C419151914D935D93EC15FD05C9F7E3
:109950002F5F3F4F2830310549F7FC01E05EFE4F95
:10996000208131813093A1142093A014FC01EE5D7D
:10997000FE4F20813181FC01EC5DFE4FF0938D0F95
:10998000E0938C0F30939F1420939E142081FC0150
:10999000EB5DFE4FF0938D0FE0938C0F2093A2149C
:1099A0002081FC01EA5DFE4FF0938D0FE0938C0F58
:1099B0002093A314623008F44AC02081FC01E95DC1
:1099C000FE4FF0938D0FE0938C0F2093A514208110
:1099D000FC01E85DFE4FF0938D0FE0938C0F209318
:1099E000A4146230A1F12081FC01E75DFE4FF093E9
:1099F0008D0FE0938C0F2093A614633041F12081EA
:109A0000FC01E65DFE4FF0938D0FE0938C0F2093E9
:109A1000A7146430E1F02081FC01E55DFE4FF09376
:109A20008D0FE0938C0F2093A814653081F0208176
:109A30003181835D9E4F90938D0F80938C0F309377
:109A4000AA142093A914663011F01FBF25C081E02D
:109A50001FBF811121C01FB7F8948DE291E0EEE79E
:109A6000F3E1DF019C011D9221503040E1F780E0DD
:109A700090E890939F1480939E142FEF2093A3144B
:109A80002FE32093A5149093AA148093A9140E9405
:109A9000AE171FBF0E94551A81E00E943E2A00E2C5
:109AA00010E076E1D72E8091F30F0E94D70E8091BF
:109AB000F30F803109F472C1992787FD90950196C3
:109AC0008F71907897FF04C00197806E9F6F019609
:109AD0008093F30F0150110931F764E1C62E66E05F
:109AE000D62E00E116E0D8018D918D010E94D70E8F
:109AF000B6E004311B07B9F700910E0110910F0178
:109B0000A0901201B090130180901001909011016B
:109B100098012A193B092819390940E050E0412CE5
:109B2000512C612C80E8782EC301B2010E94CE56E0
:109B3000209314013093150140931601509317019F
:109B40009401209530952A193B09201B310B40E0E8
:109B500050E0C301B2010E94CE5620931801309309
:109B6000190140931A0150931B0100919E1410910A
:109B70009F141093010100930001809004019090C4
:109B80000501A0900201B09003019801281939093C
:109B90002A193B0940E050E0C301B2010E94CE56B1
:109BA0002093060130930701409308015093090167
:109BB00095012095309528193909201B310B40E07B
:109BC00050E0C301B2010E94CE5620930A013093A7
:109BD0000B0140930C0150930D010E94CC220E9476
:109BE000C2216FEF8FEF0E94E0258EE697E00E9482
:109BF0008213789496EC692EAA24A39422E4722E00
:109C000030E5832E47E8942E56E1B52E9FB7F894A1
:109C10008091CB148F5F8093CB1461BA469A80FBFE
:109C2000EE24E0F8F12CEE0CFF1CEE0CFF1CE1E33F
:109C3000EE2A8E2D86958270806CA5B878B88BB888
:109C40008EB991BA9FBF10928F0F1092900F109201
:109C5000910F1092920FFFEFF093F40F04E010E0D9
:109C60000DC0992787FD909501968F71907897FD8B
:109C700001C28093F30F0150110969F08091F30F35
:109C80000E94D70E8091F30F803159F7B092F30FF5
:109C90000150110999F700E116E0D8018D918D016D
:109CA0000E94D70EC016D106C1F78091F40F8F3FE6
:109CB00011F480916C1380936C13873109F4DFC128
:109CC00081E09091A214911180E00E9492406091F5
:109CD0006C136F3F09F44FC0E62FEE0FFF0BED54EE
:109CE000F04F008111811801412C512C80916D138E
:109CF00090916E13A0916F13B091701328163906CE
:109D00004A065B06C1F120926D1330926E134092A9
:109D10006F13509270131093721300937113862F68
:109D20000E949D178823C9F0A0910E01B0910F01E8
:109D3000E0911201F09113016091100170911101F5
:109D4000CB01809590958017910708F0C1C28FEFE5
:109D50009FEF90937213809371130E94A4318091AE
:109D60006C13863109F4D3C2803109F4DBC284500C
:109D7000883008F4AAC28091CB148370823009F431
:109D80001AC2833009F4CFC1813009F4B8C10E94EE
:109D9000371C6FEF80E00E94E02538CFD092F30FA0
:109DA00099CE80E055CE0E94133E712CA12CB12C8F
:109DB00046EC542E4424439450E4652E67E8262E46
:109DC00070EE372E0FEF1FEF5FB7F89451BA469A37
:109DD00045B868B81BB81EB821BA4DE04A95F1F7EE
:109DE000000051BA469A37B867E06AB93DB845B83D
:109DF00068B81BB86EB887E481BB92E09A95F1F71A
:109E000000C026B199B18CB151BA479A422F4695FC
:109E10004370A0E82A9F90011124422B292F207122
:109E2000422B292F269526952870422B96959076C1
:109E3000492B90E0880F991F84709927482BB7EE23
:109E4000B7B9E7EFEAB9F2EEFDB95FBF41FF09C16B
:109E5000C501019662E170E0B5D2782EA82EB12C32
:109E600070928B0D2BE0271508F0F8C08FEF9FEF55
:109E700090933610809335109BEA799E912D112492
:109E800096959695892F880F890F880F472D481B27
:109E900050E0ADE1B0E1E9EFFFE080E090E00EC01E
:109EA00020E030E02D933D93118F008F01931193AB
:109EB0001387028701968630910531F08417950744
:109EC00079F72FEF3FEFEECF35E0371508F4BCC040
:109ED0008FEF9FEF90932C1080932B10809139106F
:109EE0008160809339100E940C11872D8650863036
:109EF00008F087C0AFEFBFEFB0932E10A0932D10E6
:109F0000809139108860809339100E940C114501AE
:109F1000880C991C49EF5FE0840E951E83E99BE550
:109F2000D4018D939C9388E00E949B3E6B017C0141
:109F300082EA9BEBF4019183808380E80E949B3E40
:109F4000AB01BC0110921E1010921D101092201037
:109F500010921F10109222101092211010922410B3
:109F60001092231010922610109225101092281093
:109F7000109227104C195D096E097F09C52ED62E47
:109F8000E72EFF24E7FCFA94F4E6CF16D104E104AF
:109F9000F1042CF0B3E6CB2ED12CE12CF12C2DE9E1
:109FA000C2162FEFD206E206F20634F4ADE9CA2E4D
:109FB000DD24DA94ED2CFD2CB601D7FC57C08827A0
:109FC00077FD8095982F0E94071AC701B601662772
:109FD00097FD639577278827992740E089E00E94BD
:109FE000D819F2E3FF2E8FE39CE90197F1F700C047
:109FF000000081E00E94FF0F0E94863DFA9499F7CD
:10A00000E3CE10922E1010922D1080913910877F80
:10A01000809339100E940C119BE0971508F077CFC0
:10A020004501880C991C29EF3FE0820E931E83E0C6
:10A0300094E6D4018D939C9388E00E949B3E6B0133
:10A040007C0186EC94E976CF10922C1010922B10A4
:10A05000809139108E7F8093391045CF80E090E059
:10A0600007CF42FFFDCEC5014196F4CE71956195B3
:10A070007109A5CF0197806E9F6F0196FACD60910F
:10A08000771367FD1DCE4090E10F5090E20F9201D3
:10A0900040E050E080916D1390916E13A0916F138A
:10A0A000B0917013281739074A075B0709F408CEE7
:10A0B000772767FD7095CB01880F991F860F971F33
:10A0C000880F991F880F991F805E9A4FFC01DE014F
:10A0D00011966CE001900D926A95E1F7FC011081F8
:10A0E0000181111198C0E02FEE0FFF0BE15FFC4ED4
:10A0F00051824082A0926B130E94C221E1CD6091F7
:10A1000035137091361388E10E94E12960911F1385
:10A11000709120138EE10E94E12960E070E68DE1EC
:10A120000E94E12936CE0E947E3400E010E423E054
:10A1300035E440E050EE6BE276E480913B13909181
:10A140003C130E94C1139C019093EB128093EA127E
:10A1500081E0203D37400CF080E08093EC1280914C
:10A16000491390914A13811554E0950708F4A6C04D
:10A170002091A614222309F4E4C0A0E0B0E0880FE7
:10A18000991FAA1FBB1F880F991FAA1FBB1F880FEB
:10A19000991FAA1FBB1F880F991FAA1FBB1FFD0174
:10A1A000EE0FFF1FEC5EF94F8081918190933D107F
:10A1B00080933C10EECD609111137091121389E1E0
:10A1C0000E94E12960911713709118138AE10E948F
:10A1D000E1298091CF0F9091D00F4091E8125091DA
:10A1E000E912662757FD6095762F480F591F611DAC
:10A1F000711D77FD88C0CB01BA016115710531E091
:10A200008307910524F06FEF7FEF80E090E08BE112
:10A210000E94E129BECD133008F06CCF4D863E87F9
:10A220004F87588B0E94A813FE01359660E070E0BE
:10A23000CB012D853E854F855889A191B191AB2BDE
:10A2400049F06F5F7F4F8F4F9F4F643071058105DD
:10A25000910599F7A8D01C01552437FC5094452C42
:10A260008091731390917413A0917513B09176132C
:10A27000281639064A065B0671F0F1013296EE0F98
:10A28000FF1F21E030E02C0F3D1FE20FF31F808104
:10A2900091810E948213113009F04DC0E02FFF27F9
:10A2A000E7FDF095EB50FD4E208220927313309223
:10A2B000741340927513509276131CCF8FEF9FEF5B
:10A2C00090933D1080933C1064CD0E94492053CD63
:10A2D0000617170708F444C0CD018E1B9F0B081703
:10A2E000190708F040C0A2019101261B370B410954
:10A2F000510960911401709115018091160190919E
:10A30000170151D026CD40E050E0BA0174CF6091E2
:10A31000DF0F7091E00F21E042E080E090E00E94CA
:10A32000AE1D29CD0E943C3121E041E060E070E0AB
:10A330000E94AE1D20CDB201A101802F0E94B01F4E
:10A34000B4CF00E010E02AEF33E440E050EE6BEAD7
:10A3500076E40E94C11390933D1080933C1019CD78
:10A3600080E090E0F6CCCF018A0F9B1F8017910709
:10A3700018F080E090E8EDCCA2019101281B390B88
:10A3800041095109609118017091190180911A01D8
:10A3900090911B0108D09058DCCCF4D4B7FF0895FD
:10A3A000821B930B0895DB018F939F93ACD4BF91D5
:10A3B000AF91A29F800D911DA39F900DB29F900D14
:10A3C0001124089597FB072E16F4009406D077FD0C
:10A3D00008D0A9D407FC05D03EF4909581959F4FF5
:10A3E0000895709561957F4F08955058BB27AA270F
:10A3F0000ED0F1C1BAD130F0BFD120F031F49F3F7F
:10A4000011F41EF48AC10EF4E095E7FB80C1E92F38
:10A4100004D280F3BA17620773078407950718F010
:10A4200071F49EF51CC20EF4E0950B2EBA2FA02DF0
:10A430000B01B90190010C01CA01A0011124FF27F1
:10A44000591B99F0593F50F4503E68F11A16F040EC
:10A45000A22F232F342F4427585FF3CF46953795EB
:10A460002795A795F0405395C9F77EF41F16BA0BB0
:10A47000620B730B840BBAF09150A1F0FF0FBB1F5E
:10A48000661F771F881FC2F70EC0BA0F621F731FA7
:10A49000841F48F4879577956795B795F7959E3F04
:10A4A00008F0B3CF9395880F08F09927EE0F979592
:10A4B0008795089508D108F481E0089565D1E39562
:10A4C0009BC10CD088C158D140F04FD130F021F45D
:10A4D0005F3F19F01CC15111C3C11FC19ED198F338
:10A4E0009923C9F35523B1F3951B550BBB27AA2715
:10A4F00062177307840738F09F5F5F4F220F331F87
:10A50000441FAA1FA9F333D00E2E3AF0E0E830D052
:10A5100091505040E695001CCAF729D0FE2F27D055
:10A52000660F771F881FBB1F261737074807AB0723
:10A53000B0E809F0BB0B802DBF01FF2793585F4F98
:10A540002AF09E3F510568F0E2C08AC15F3FECF3FC
:10A55000983EDCF3869577956795B795F7959F5F5D
:10A56000C9F7880F911D9695879597F90895E1E0B1
:10A57000660F771F881FBB1F621773078407BA0710
:10A5800020F0621B730B840BBA0BEE1F88F7E0956B
:10A59000089519F40EF0BBC062C1BFC046D1C8F324
:10A5A0009638C0F707F80F92E8942BE33AEA48EBA5
:10A5B0005FE7DED10F920F920F924DB75EB70F9209
:10A5C00096D1ECEAF0E0ACD04F915F91EF91FF9122
:10A5D000E595EE1FFF1F49F0FE57E0684427EE0F98
:10A5E000441FFA95E1F74195550B4DD10F9007FEA9
:10A5F00041C108951AD188F09F5790F0B92F99273B
:10A60000B751A0F0D1F0660F771F881F991F1AF07D
:10A61000BA95C9F712C0B13081F021D1B1E00895E7
:10A620001EC1672F782F8827B85F39F0B93FCCF368
:10A63000869577956795B395D9F73EF49095809573
:10A64000709561957F4F8F4F9F4F0895E89409C093
:10A6500097FB3EF490958095709561957F4F8F4F55
:10A660009F4F9923A9F0F92F96E9BB279395F6956B
:10A67000879577956795B795F111F8CFFAF4BB0FE9
:10A6800011F460FF1BC06F5F7F4F8F4F9F4F16C04D
:10A69000882311F096E911C0772321F09EE8872FD7
:10A6A000762F05C0662371F096E8862F70E060E093
:10A6B0002AF09A95660F771F881FDAF7880F96950C
:10A6C000879597F90895990F0008550FAA0BE0E8B0
:10A6D000FEEF16161706E807F907C0F01216130664
:10A6E000E407F50798F0621B730B840B950B39F4A4
:10A6F0000A2661F0232B242B252B21F408950A260A
:10A7000009F4A140A6958FEF811D811D089597F949
:10A710009F6780E870E060E008959FEF80EC089507
:10A72000DF93CF931F930F93FF92EF92DF927B0102
:10A730008C01689405C0DA2EEF0118D1FE01E8946F
:10A74000A5912591359145915591AEF3EF015FDECD
:10A75000FE019701A801DA9479F7DF90EF90FF905E
:10A760000F911F91CF91DF91089500240A9416163E
:10A77000170618060906089500240A9412161306EF
:10A78000140605060895C9CF50D0E8F3E894E0E038
:10A79000BB279F57F0F02AED3FE049EC06C0EE0FD3
:10A7A000BB0F661F771F881F28F0B23A6207730736
:10A7B000840728F0B25A620B730B840BE3959A95C9
:10A7C00072F7803830F49A95BB0F661F771F881F89
:10A7D000D2F7904870C1092E0394000C11F488231D
:10A7E00052F0BB0F40F4BF2B11F460FF04C06F5F49
:10A7F0007F4F8F4F9F4F0895EF93E0FF06C0A2EA6F
:10A800002AED3FE049EC5FEB02DEE5DF0F900394B9
:10A8100001FC9058E4EDF0E05AC157FD9058440F08
:10A82000551F59F05F3F71F04795880F97FB991FAF
:10A8300061F09F3F79F0879508951216130614066C
:10A84000551FF2CF4695F1DF08C0161617061806F9
:10A85000991FF1CF86957105610508940895E894D4
:10A86000BB2766277727CB0197F908952CDF08F4DB
:10A870008FEF08959B01AC0160E070E080E89FE3FA
:10A8800020CE45CF16C1D1DFE8F39923D9F3940F39
:10A89000511DBBF39150504094F059F0882332F091
:10A8A000660F771F881F91505040C1F79E3F51059A
:10A8B00044F7880F911D9695879597F908955F3F06
:10A8C000ACF0983E9CF0BB27869577956795B79539
:10A8D00008F4B1609395C1F7BB0F58F711F460FF0E
:10A8E000E8CF6F5F7F4F8F4F9F4FE3CFB9CFFA0114
:10A8F000DC01AA0FBB1F9B01AC01BF5728F4222724
:10A900003327442750781FC0B75188F4AB2F002459
:10A91000469537952795011CA395D2F3002069F041
:10A92000220F331F441FB395DAF30DD05ECD613093
:10A930007105A0E88A07B94630F49B01AC0166278F
:10A94000772788279078309621F0208331834283BF
:10A95000538308950BD03FCF08DF28F00DDF18F0A8
:10A96000952309F0D4CED9CE11247ACF56DFA0F3A7
:10A97000959FD1F3950F50E0551F629FF001729F94
:10A98000BB27F00DB11D639FAA27F00DB11DAA1FB3
:10A99000649F6627B00DA11D661F829F2227B00D00
:10A9A000A11D621F739FB00DA11D621F839FA00D8B
:10A9B000611D221F749F3327A00D611D231F849FDB
:10A9C000600D211D822F762F6A2F11249F57504032
:10A9D0008AF0E1F088234AF0EE0FFF1FBB1F661FCD
:10A9E000771F881F91505040A9F79E3F510570F086
:10A9F0008ECE36CF5F3FECF3983EDCF386957795AD
:10AA00006795B795F795E7959F5FC1F7FE2B880F80
:10AA1000911D9695879597F90895FA01EE0FFF1FFE
:10AA200030962105310599F16115710561F4803881
:10AA3000BFE39B0749F168949038810561F0803845
:10AA4000BFEF9B0741F0992342F5FF3FE105310538
:10AA5000210511F1E8940894E795D901AA2329F476
:10AA6000AB2FBE2FF85FD0F310C0FF5F70F4A69538
:10AA7000E0F7F73950F019F0FF3A38F49F779F93D9
:10AA80000CD00F9007FC905808953EF046CE60E041
:10AA900070E080E89FE308954FE79F775F934F93BF
:10AAA0003F932F932AD02F913F914F915F9152DF87
:10AAB00075CD9F3F31F0915020F48795779567953C
:10AAC000B795880F911D9695879597F908959F934F
:10AAD0008F937F936F93FF93EF939B01AC013ADFCA
:10AAE000EF91FF911DDE2F913F914F915F9132CFFA
:10AAF0000EF0DFCF12CE68940ACE97DEC8F399230A
:10AB0000D1F3C6F3DF93CF931F930F93FF92C92F17
:10AB1000DD2788232AF02197660F771F881FDAF731
:10AB200020E030E040E85FEB9FE3883920F0803E92
:10AB300030F021968F775ADCE2EFF0E003C056DC6C
:10AB4000EFE1F1E0EDDD8B01BE01EC01FB2E6F5773
:10AB500071097595771F880B990B7ADD28E132E72B
:10AB600041E35FE303DFAF2D9801AE01FF900F914A
:10AB70001F91CF91DF914BDC2ECEFB01DC0104C095
:10AB80008D910190801921F441505040C8F7881BE5
:10AB9000990B0895FB01DC0102C001900D92415018
:10ABA0005040D8F708956817790768F4FB01DC0175
:10ABB000E40FF51FA40FB51F02C002900E92415082
:10ABC0005040D8F70895E6CFDC0101C06D934150A5
:10ABD0005040E0F70895FB01DC010D900020E9F7FB
:10ABE000119701900D920020E1F70895FB01DC011F
:10ABF00001900D920020E1F708958F929F92AF92FD
:10AC0000BF92CF92DF92EF92FF92CF93DF93EC014E
:10AC1000688179818A819B81611571058105910522
:10AC200021F464E279ED8BE597E02DE133EF41E02B
:10AC300050E08DD049015A019B01AC01A7EAB1E473
:10AC400062D06B017C01ACEEB4EFA501940167D03A
:10AC5000C60ED71EE81EF91EF7FE06C081E0C81A10
:10AC6000D108E10880E8F80AC882D982EA82FB822A
:10AC7000E894F7F8B601C701DF91CF91FF90EF900C
:10AC8000DF90CF90BF90AF909F908F900895B5CFF9
:10AC90008CE191E0B2CF60931C0170931D01809311
:10ACA0001E0190931F010895FB019F01E89442301B
:10ACB000BCF04532ACF44A3029F497FB1EF4909571
:10ACC00081959F4F642F77272ED0805D8A330CF0BB
:10ACD000895D8193CB010097A9F716F45DE251934A
:10ACE0001082C90100C0DC01FC01672F719177233C
:10ACF000E1F7329704C07C916D9370836291AE1737
:10AD0000BF07C8F308953ED0A59F900DB49F900D46
:10AD1000A49F800D911D11240895B7FFF4CFF3DF98
:10AD2000821B930B0895AA1BBB1B51E107C0AA1FEE
:10AD3000BB1FA617B70710F0A61BB70B881F991FDC
:10AD40005A95A9F780959095BC01CD010895052EDF
:10AD500097FB16F4009406D057FD0CD01FD007FCCB
:10AD600009D07EF490958095709561957F4F8F4FB7
:10AD70009F4F089550954095309521953F4F4F4FE7
:10AD80005F4F0895A29FB001B39FC001A39F01D060
:10AD9000B29F700D811D1124911D0895A1E21A2EFC
:10ADA000AA1BBB1BFD010DC0AA1FBB1FEE1FFF1F6F
:10ADB000A217B307E407F50720F0A21BB30BE40BBF
:10ADC000F50B661F771F881F991F1A9469F7609506
:10ADD0007095809590959B01AC01BD01CF010895C0
:04ADE000F894FFCF15
:10ADE40000809001000C00000000000000000080C2
:10ADF4000000000800000000000000000100000046
:10AE040000006207640E3415D21B41228128942E5F
:10AE14007B34383ACB3F37457B4A994F9254675934
:10AE24001A5EAB621A676A6B9B6FAD73A2777B7B0A
:10AE3400387FD9826186CF89258D629088939896D0
:10AE44009199759C449FFFA1A6A43AA7BBA92AACDB
:10AE540088AED5B011B33DB559B766B964BB54BD1E
:10AE640036BF0BC1D2C28CC43AC6DCC772C9FDCA94
:10AE74007CCCF1CD5BCFBBD011D25ED3A1D4DBD5DA
:10AE84000CD734D854D96DDA7DDB85DC86DD80DEE1
:10AE940073DF5FE044E123E2FCE2CEE39BE461E59F
:10AEA40022E6DEE695E746E8F2E89AE93DEADBEADF
:10AEB40074EB0AEC9BEC28EDB1ED36EEB8EE36EF10
:10AEC400B0EF27F09AF00BF178F1E2F149F2ADF22C
:10AED4000EF36DF3C9F322F479F4CDF41FF56FF595
:10AEE400BCF507F651F698F6DDF620F761F7A0F702
:10AEF400DEF71AF854F88DF8C4F8F9F82DF95FF96B
:10AF040090F9C0F9EEF91BFA47FA71FA9BFAC3FA01
:10AF1400EAFA10FB35FB58FB7BFB9DFBBEFBDEFB1B
:10AF2400FDFB1BFC38FC55FC70FC8BFCA5FCBFFC3A
:10AF3400D8FCF0FC07FD1EFD34FD49FD5EFD72FDED
:10AF440086FD99FDABFDBDFDCFFDE0FDF0FD01FEED
:10AF540010FE1FFE2EFE3CFE4AFE58FE65FE72FEEB
:10AF64007EFE8AFE96FEA2FEADFEB7FEC2FECCFEBB
:10AF7400D6FEE0FEE9FEF2FEFBFE04FF0CFF14FF2A
:10AF84001CFF23FF2BFF32FF39FF40FF47FF4DFF1C
:10AF940053FF59FF5FFF65FF6BFF70FF75FF7BFF7A
:10AFA40080FF84FF89FF8EFF92FF96FF9BFF9FFF28
:10AFB400A3FFA7FFAAFFAEFFB1FFB5FFB8FFBBFF1A
:10AFC400BFFFC2FFC5FFC8FFCAFFCDFFD0FFD2FF3E
:10AFD400D5FFD7FFDAFFDCFFDEFFE0FFE3FFE5FF8D
:10AFE400E7FFE9FFEAFFECFFEEFFF0FFF1FFF3FFFD
:10AFF400F5FFF6FFF8FFF9FFFBFFFCFFFDFFFFFF86
:10B004000000EE01DA03C305A9078C096C0B4A0D95
:10B01400250FFD10D212A414741641180B1AD31B59
:10B02400981D5A1F1A21D72291244926FE27B12997
:10B03400612B0E2DB92E62300832AB334D35EB3611
:10B044008738213AB93B4E3DE03E7140FE418A4388
:10B0540013459A461F48A149224B9F4C1B4E944FBF
:10B064000C518152F4536455D3563F58A959115B7E
:10B07400775CDB5D3D5F9C60FA615663AF64076695
:10B084005C67B068016A516B9E6CEA6D346F7B70CB
:10B09400C171057347748775C57602783C79757AF2
:10B0A400AC7BE17C147E457F7580A381CF82F983DC
:10B0B400218548866D879188B289D28AF18B0D8D5E
:10B0C400288E418F59906F9183929693A794B69549
:10B0D400C496D197DB98E599EC9AF29BF79CFA9D7C
:10B0E400FB9EFB9FFAA0F7A1F2A2ECA3E5A4DCA5CA
:10B0F400D2A6C6A7B9A8AAA99AAA88AB76AC61AD0C
:10B104004CAE35AF1CB003B1E7B1CBB2ADB38EB426
:10B114006EB54CB629B705B8DFB8B8B990BA67BBF5
:10B124003CBC10BDE3BDB4BE85BF54C022C1EEC15A
:10B13400BAC284C34DC415C5DCC5A2C666C729C836
:10B14400ECC8ADC96DCA2BCBE9CBA5CC61CD1BCE68
:10B15400D4CE8DCF44D0FAD0AFD162D215D3C7D3D9
:10B1640078D427D5D6D584D630D7DCD786D830D96D
:10B17400D9D980DA27DBCCDB71DC15DDB7DD59DE0C
:10B18400FADE9ADF39E0D7E074E110E2ACE246E39C
:10B19400DFE378E410E5A6E53CE6D1E665E7F9E708
:10B1A4008BE81CE9ADE93DEACCEA5AEBE7EB74EC39
:10B1B40000ED8AED14EE9EEE26EFAEEF35F0BBF017
:10B1C40040F1C4F148F2CBF24DF3CEF34FF4CFF497
:10B1D4004EF5CCF54AF6C7F643F7BEF739F8B3F89F
:10B1E4002CF9A5F91DFA94FA0AFB80FBF5FB6AFC1D
:10B1F400DDFC50FDC3FD34FEA5FE16FF85FFF4FF04
:10B20400001D8E07000000000000000002009407EB
:10B214009C07A507AD070000001AB6070000000050
:10B2240000000000001BBE0700000000000000003A
:10B234000019C60700000000000000000202CE074B
:10B24400D607DF07E807F0070114F8070809010823
:10B254000508090800160D080000000000000000A1
:10B26400001C1308000000000000000000171A086A
:10B274000000000000000000001D8E070000000018
:10B2840000000000020122082A0832082B082D08B9
:10B29400010A34083C084008000000000205450883
:10B2A4004D083C0840085108011756085E0862081A
:10B2B4000000000002036608D607DF07E807F0076E
:10B2C40002046E0877087B087F0883080112870848
:10B2D4008C083C08400800000116910897089C0857
:10B2E400A10800000018A5080000000000000000EC
:10B2F40001101E1DC000A8009000800060004800DE
:10B3040030002400180012000C000900060004009C
:10B3140003000200080C080A0808080808080808BE
:10B32400080A080C0C0000000000080C0A0A0A0AAB
:10B334000A0C0C08000000000000000000000000DF
:10B3440000000000000000000000000000000000F9
:10B3540000000000003022366D247D20390F76462F
:10B36400104010523F065B4F666D7D077F6F484863
:10B37400614843277B777F393F79713D76060E76A6
:10B384003837373F733F776D783E3E7E76665B395C
:10B39400640F230802777C585E79716F74040C740F
:10B3A4003837545C7367506D781C1C7E766E5B393D
:10B3B400300F010001010101010101010103020635
:10B3C400020101010001020402030201020174727C
:10B3D400616E7370203D20000000000000007509BC
:10B3E4007A097E09820986098A098E0992099609D1
:10B3F4009A099E09A309A809AD09B209B709BC09AC
:10B40400FCFDFE010204081020408000FFFFFFFF46
:10B41400FF1E00181D0C0D1F01020304050607087A
:10B42400090A0B191B1A1CFFFFFFFFFFFFFFFF0296
:10B4340003020000010001010101010001010037C4
:10B4440056656F7C878B8F949AA4B0B9BFD2476C32
:10B4540069476C69277320503630302075706772E5
:10B464006164652056657220322E3039390073705C
:10B47400656564006C666F207368700070756C732A
:10B484002D74726900726E642D73696E006E6F693B
:10B49400732D736177005669622073706400566976
:10B4A4006220616D74006D6F6420646C7900616D5D
:10B4B400702073687000666173742D65787000661F
:10B4C4006173742D6C696E00736C6F2D65787000F8
:10B4D400736C6F2D6C696E0062656E6420746774A2
:10B4E4000056636F0056636600566F6C00676C69A4
:10B4F400646500646574756E6500616D70205665E1
:10B504006C006C666F207467740061620061622D68
:10B51400566361006C666F2072616E006C6F770019
:10B5240068696768006D6F642072616E006D696E92
:10B534000066756C6C006D6F6420746774006C66D3
:10B544006F005669620066696C20736870006265FA
:10B554006E642072616E00326E6400337264003572
:10B564007468004F6374007072696F006C61737467
:10B5740000706974636800667265650073656D695F
:10B58400006F63740066696C2056656C0062656EBA
:10B594006465722063616C696272617465640070D1
:10B5A4007265736574732064756D706564002072D0
:10B5B400656376002073656E640070726573732032
:10B5C400616761696E20666F722062656E64657280
:10B5D4002063616C6962726174696F6E0056632DD9
:10B5E400206F6E0056632D206F666600707265735F
:10B5F4007320616761696E20746F2064756D7020BB
:10B604007072657365747300496E742073796E6328
:10B61400004D6964692073796E63007461706520FC
:10B6240073796E63007370726561642000202F204B
:10B63400566366206C696D200070726573732061B7
:10B644006761696E20666F7220626173696320703E
:10B6540061746368006F6D6E6900636831006368CC
:10B6640032006368330063683400636835006368DC
:10B6740036006368370063683800636839006368BC
:10B6840031300063683131006368313200636831FE
:10B6940033006368313400636831350063683136E0
:02B6A4000000A4
:020000021000EC
:10E000002F923F924F925F926F927F928F929F9248
:10E01000AF92BF92CF92DF92EF92FF920F931F9336
:10E02000CF93DF93CDB7DEB728970FB6F894DEBF56
:10E030000FBECDBF2FEF31EE44E0215030404040C5
:10E04000E1F700C00000F89414B817B81AB81DB86A
:10E0500010BA15B890EE98B91BB81EB883EE81BB04
:10E060002FEF24B997B947E04AB99DB980BB36EC88
:10E0700031BB469A97B94AB99DB915B880E888B9B5
:10E080001BB81EB8F7E4F1BB62E06A95F1F700C077
:10E0900086B189B18CB131BB479AE7EEE7B977EF2A
:10E0A0007AB962EE6DB931BB469AA1E0A5B982E4B6
:10E0B00088B91BB81EB887E881BB8DE08A95F1F757
:10E0C000000031BB469A97B94AB99DB9A5B920E479
:10E0D00028B91BB82EB9F1BBB2E0BA95F1F700C070
:10E0E00086B159B1BCB131BB479AE7B97AB96DB9BC
:10E0F000BDE0BA95F1F7000031BB469A97B94AB92D
:10E100009DB9A5B928B91BB82EB9F1BBF2E0FA95B3
:10E11000F1F700C026B199B14CB131BB479AE7B9CC
:10E120007AB96DB93DE03A95F1F70000422F469576
:10E13000437060E8269F90011124242B392F307101
:10E14000322B292F269526952870232B969590768D
:10E15000922B907C21E0903C09F020E0382F3695FE
:10E160003370A0E88A9FC0011124832B952F9071F2
:10E17000982B852F869586958870982B852F869568
:10E180008076982B907C81E0903C09F080E082239F
:10E1900009F4EEC186EC81BB469A21E025B990E4F2
:10E1A00098B99BB91EB897E891BBBAE0BA95F1F758
:10E1B00000C081BB469A25B934E438B930E73BB991
:10E1C00032E23EB991BBEAE0EA95F1F700C081BBCB
:10E1D000469A25B922E428B920E52BB920EC2EB9BE
:10E1E00091BBFAE0FA95F1F700C081BB469A15B8E9
:10E1F00026E828B923E02BB91EB891BBAFE9BFE0F0
:10E200001197F1F700C0000081BB469A15B823E8CA
:10E2100028B923E12BB922E02EB991BBBAE0BA9517
:10E22000F1F700C081BB469A20EE27B997E09AB972
:10E230002DB915B870E878B99BB91EB867E461BB11
:10E24000E2E0EA95F1F700C036B139B13CB181BBEB
:10E25000479A57EE57B947EF4AB932EE3DB9F5E064
:10E26000FA95F1F7000081BB469A27B99AB92DB902
:10E2700015B878B99BB990E29EB961BB22E02A95A6
:10E28000F1F700C096B199B19CB181BB479A57B9DB
:10E290004AB93DB935E03A95F1F7000099249394D5
:10E2A0000F2EFEE72F2EF8E13F2EF02D0F2EFEE76A
:10E2B0004F2EF9E15F2EF02D88248394BED499234C
:10E2C0000CF441C1803F9105C9F7B7D4892B09F0FF
:10E2D0003AC1B3D48136910509F035C1AED4469721
:10E2E00009F031C1AAD48B36910509F02CC1A5D40F
:10E2F0007C0199230CF427C1682F80E090E080D442
:10E300008C01E894E7F8FF24F694FE2CEE24F794B1
:10E31000E79493D46C0199230CF415C1682FC801BC
:10E320006FD48C01E894C7F8DD24EC28FD28E114B3
:10E3300041E0F40621F0EF2809F407C104C17DD4BF
:10E340006C0199230CF4FFC0682FC80159D48C01CB
:10E3500074D45C0199230CF4F6C0682FC80150D422
:10E3600098878F83810169D47C0199230CF483C041
:10E37000682F8F81988544D498878F83C7018F77C2
:10E3800099279A83898359D47C0199230CF473C00B
:10E39000682F8F81988534D498878F83D701AF7782
:10E3A000BB27BC83AB8349D47C0199230CF463C0A5
:10E3B000682F8F81988524D498878F83F701EF7712
:10E3C000FF27FE83ED8339D47C0199230CF453C0DD
:10E3D000682F8F81988514D498878F833701E894AC
:10E3E00067F877242AD47C0199230CF444C0682F61
:10E3F0008F81988505D498878F83F8013397C7015B
:10E400009695982F8827979587952981822B8083C9
:10E41000F8013297C7018270992700249695879555
:10E420000794969587950794982F802D3B81832B91
:10E430008083F8013197C70184709927880F991F4D
:10E4400082959295907F9827807F98274D81842B85
:10E450008083C7018870992782959295907F98272D
:10E46000807F98278629D8018C930C5F1F4F041555
:10E47000150509F078CFE1D399230CF464C08C0121
:10E48000102F0027110FD9D399230CF45CC08F777C
:10E490009927880F991F880F991F082B192BCDD307
:10E4A00099230CF450C083709927082B192BEF8106
:10E4B000F8850E171F0709F046C0BFD3873F9105A7
:10E4C00009F041C0990CFFE3F91508F4982C26ECEB
:10E4D00021BB469A892D880F392D3695282F267015
:10E4E0002064992D991F9927991F292B992D907197
:10E4F000482F440F4072942B807C982B832F82707E
:10E50000806285B828B99BB98EB937E831BB4AE03B
:10E510004A95F1F700C0B5016F777727C6018F776D
:10E5200099279695982F882797958795682B792B0B
:10E53000CB01A0E0B0E06627782F892F9A2F4BE718
:10E5400058E15ED5BBCE89E701C08DE696EC91BB64
:10E55000469A982F9071906E86958270806221E025
:10E5600025B922E428B99BB98EB987E881BBFFCFD2
:10E5700028960FB6F894DEBF0FBECDBFDF91CF91C6
:10E580001F910F91FF90EF90DF90CF90BF90AF90D1
:10E590009F908F907F906F905F904F903F902F90C3
:02E5A0000895DC
:10EC00009C013627032E0294802D8F708327632F5B
:10EC10006025660F607E8627602D6327607F66957E
:10EC2000032E000C661F3695369536953F713627B4
:10EC30003227282F822F932F089545E04A95F1F728
:10EC40000000349B04C000C000C03499FCCF86ECA7
:10EC500081BB469A20EE27B997E09AB92DB915B82D
:10EC600020E828B99BB91EB897E491BB52E05A95A9
:10EC7000F1F700C096B129B13CB181BB479A87EE4C
:10EC800087B987EF8AB982EE8DB985E08A95F1F769
:10EC90000000392F3695337040E8949FC00111244D
:10ECA000832B922F9071892B922F96959695987021
:10ECB000892B26952076282B217B213809F040C00E
:10ECC00026EC21BB469A90EE97B987E08AB99DB9A8
:10ECD00015B890E898B98BB980E28EB987E481BB0A
:10ECE00052E05A95F1F700C036B199B14CB121BB51
:10ECF000479A87EE87B987EF8AB982EE8DB985E0AA
:10ED00008A95F1F70000832F8695837050E8359F30
:10ED100090011124282B892F8071282B892F86950B
:10ED200086958870282B96959076292B50E0CA01FD
:10ED3000880F991F84709927822B282F30E002C0FA
:0AED40002FEF3FEF822F932F08956D
:10F000008F929F92AF92BF92CF92EF92FF92CF9347
:10F01000DF93EA01CFB6F894F999FECF23E0FB0124
:10F0200080935B002093570010D707B600FCFDCFFC
:10F03000DE01B3954B015C0121E04881F980E12CB0
:10F04000F701E40FF11DAF0122960A01F401A0922D
:10F050005B0020935700F9D61124F2E08F0E911C2B
:10F06000A11CB11CAC17BD0741F725E0FB01809343
:10F070005B0020935700E9D607B600FCFDCF81E185
:10F0800080935700E2D6CFBEDF91CF91FF90EF90F3
:0CF09000CF90BF90AF909F908F9008959C
:00000001FF
